:100000000C9437080C945F080C945F080C945F08FC
:100010000C945F080C945F080C945F080C945F08C4
:100020000C945F080C945F080C94F8280C946729D2
:100030000C945F080C945F080C945F080C945F08A4
:100040000C945F080C945B2C0C945F080C945F0874
:100050000C945F080C945F080C945F080C94992B27
:100060000C945F080C945F080C945F080C945F0874
:100070000C945F080C945F080C945F080C945F0864
:100080000C94E32B0C945F080C945F080C945F08AD
:100090000C945F080C945F080C945F080C945F0844
:1000A0000C945F080C945F080C945F08084AD73BD7
:1000B0003BCE016E84BCBFFDC12F3D6C74319ABD37
:1000C00056833DDA3D00C77F11BED9E4BB4C3E915B
:1000D0006BAAAABE000000803F0000000000007074
:1000E0000100C0000C00CAA77C0A42F55508534223
:1000F00048195EF551120030000000274500409479
:100100001C0014F3190504F111042004000004413B
:10011000100400040000104208015E14450F40F076
:1001200001005955551351555D0D8C927C0857555A
:10013000550D5E55550D51520C015E55550F5655D6
:10014000550F00A0000000A4000000C2280080A2FB
:1001500028008062080040500D005E7455079C9294
:10016000241F5F555D0D9C1445115F1425075F55D5
:1001700055115F5114015E54551D1F41101F40F46D
:100180004500100421071F41181D1F0441105EF097
:10019000041F9C10041F5E54450F5F9214035ED42D
:1001A000451F5F92341B5655550D41F005011F0444
:1001B00021071F4208011FE4410F1743181D07C103
:1001C000090151564D1100F0450000F0010040F4C6
:1001D000010080100C0010044110050115012501DB
:1001E000370149015D01720188019F01B801D20107
:1001F000EE010B022A024B026E029302BA02E402E3
:1002000010033E037003A403DC0316045404960495
:10021000DC0426057505C80520067D06E0064807AE
:10022000B7072D08A9082D09B9094D0AEA0A900B4C
:10023000400CFA0CC00D910E6F0F5A1053115A1248
:1002400072139A14D31520178018F519801B221DDC
:10025000DE1EB420A622B524E4263429A72B402E86
:100260000031080809090A0B0B0C0D0E0E0F1011B6
:100270001213141617181A1B1D1F20222427292BAE
:100280002E3134373A3D4145494E52575C62686ED3
:10029000747B838A939BA5AEB9C4CFDCE9F70001D8
:1002A00002030406080C00F4F8FAFCFDFEFF3E47CA
:1002B0006B6D6D413E3E41555551653E000306094B
:1002C0000C0F1215181C1F2225282B2E30333639FF
:1002D0003C3F414447494C4E515355585A5C5E602F
:1002E000626466686A6C6D6F707273757677787920
:1002F0007A7B7C7C7D7E7E7F7F7F7F7F80904800C5
:1003000064904A0064904C0064904D0064904F00EB
:10031000C880F0D02869281B28367F775514080834
:10032000082A6B7F3E2A081C3E36637F6341081C07
:10033000495D7F2A49143E7F6B632214775D551C0B
:100340003E3622000000C0F0F0F8F8F8F0F0C000EF
:1003500000000000000107070F0F0F070701000052
:100360000000E0F8FCFCFEFEFEFEFEFCFCF8E000F7
:1003700000030F1F1F3F3F3F3F3F1F1F0F0300E0C2
:10038000F8FCFEFEFF3F3F3FFFFEFEFCF8E0030FE0
:100390001F3F3F7F7E7E7E7F3F3F1F0F03E0F8FCC5
:1003A000FE3E1F0F0F0F1F3EFEFCF8E0030F1F3F26
:1003B0003E7C7878787C3E3F1F0F03E0F81C0E06E9
:1003C0000303030303060E1CF8E0030F1C38306020
:1003D0006060606030381C0F03E018040202010105
:1003E00001010102020418E0030C102020404040EB
:1003F00040402020100C035449544C4500524554B1
:10040000525900FCFEFE063E3E3C00E0F0F030F0AB
:10041000F0E000F0F0F020F0F0E020F0F0E000F08C
:10042000F0F020F0F0E000FEFEFE00E0F0F0B0F0B2
:10043000F0E000FCFCFC3000E0F0F0B0F0F0E00098
:10044000E0F0F020FEFEFE00FEFEFE1F3F3F303FCC
:100450001F0F001F3F3F303F3F1F003F3F3F003F08
:100460003F3F003F3F3F007F7F7F103F3F1F003FE8
:100470003F3F001F3F3F313D3D1D003F3F3F3000AC
:100480001F3F3F313D3D1D001F3F3F103F3F3F009D
:100490003B3B3BFEFEFEC6C600E0F0F030F0F0E075
:1004A00000F6F6F600FEFEFE00E0F0F0B0F0F0E040
:1004B00000E0F0F020FEFEFE000000000000000062
:1004C000003F3F3F0000001E3E3E133F3F3F003FC6
:1004D0003F3F003F3F3F001F3F3F313D3D1D001F5D
:1004E0003F3F103F3F3F003838003838003838FE73
:1004F000FEFEC6FEFE7C00E0F0F0B0F0F0E000E0B2
:10050000F0F030F0F0E000E0F0F020FEFEFE0070D1
:10051000F0F08000F0F07000DCDEDE86FEFCF83FDC
:100520003F3F003F3F3F001F3F3F313D3D1D001E0D
:100530003E3E133F3F3F001F3F3F103F3F3F000005
:10054000637F7F787F1F00003B3B3B0101010090F0
:1005500051002880002890560028800028905A00DA
:1005600028800028E3F0DE945000089447000894A7
:100570004C000894430008E480F04241434B20546F
:100580004F205449544C4500524554525900434F52
:100590004E54494E554500550E644F0F5DDD9C5D30
:1005A000000A9C51000AE380F0904C000A90490038
:1005B0000A80F043414E43454C004F4B005041549C
:1005C0005445524E3A004F424E2D59313320564534
:1005D0005220302E313100C0C6CFDFFFFB73037CC9
:1005E000FEFFC7E3FF7F3E00FFFFFF1B1B1B030057
:1005F0000303FFFFFF030300000000000000008072
:1006000080808000000000000000000000000080EA
:10061000E0F058AC56AB55AB5500FF0101010202AA
:10062000040810608000003FFFAA55AA55AA55AAE9
:1006300055A85FAC5CAC5CAC5CAC5C0CCF3C000027
:10064000000103060D1A152A252A252A252215122E
:1006500009040201000000FFFF57AB57AB57AB572F
:10066000AB03FF808080000000000000000000FF5E
:10067000FF55AA55AA55AA55AA00FF00000001017E
:1006800002040830C000001F7FD5AA55AA55AA55FC
:10069000AA54AF56AE56AE56AE562E86671E000012
:1006A00000000103060D0A151215121512110A0990
:1006B000040201000000000000000000008080C073
:1006C000C0C0C0808080000000000000000000C0AA
:1006D000F078AC56AB55AA55AA00FF000000010106
:1006E00002040830C00000FFFF55AA55AA55AA55BC
:1006F000AA00FFFEAE56AE56AE56AE5607FE001F1F
:10070000171512151215121512101F1712151215A2
:1007100012151215101F000000A040A00028104460
:1007200038827C007C8ED6DADA827C003838003859
:100730007CFE0000000000240027002A002D00306D
:100740000000000000250028002B002E00310004CE
:1007500008020110408040102040804080080204C0
:10076000018040201002011080102040402004042D
:10077000040404030405020202020403020202024A
:100780000606060606060404020202040400009996
:100790001408153F13D3130000AE1FEB1EC91B87AF
:1007A000184352454449540053455454494E475305
:1007B000004E455720424154544C45005245545236
:1007C0005900455849540044455445435420454434
:1007D0004745004C454420424C494E4B0050415443
:1007E0005445524E00444946464943554C545900DD
:1007F0000C0E06030303060E040C0E1E0F0F0F0E45
:100800000E040C0E1E1F1F1F0E0E0470FC0E06039E
:10081000030370FC7E3E0F0F0F70FC7E3E3F1F0FE8
:10082000000000000000000000807E1FBC78E0C0D7
:10083000C080808080404020B058AC5CB878F0E048
:10084000C000000000804020A0108847A050AA559A
:10085000AAF50BE7060C0A1C7AF5FAFD7E030101E6
:1008600002050B070E314994BA7DFEEDC607070954
:1008700012254A558A952B563050B87FFFFFFCE071
:100880000000000000000000000000010205070356
:1008900000000000000000000101020408152A55B4
:1008A0006FDFFF78000000004F4646004F4E2000EB
:1008B00052414E444F4D2000535045434946590044
:1008C000504C41592054494D4500504C415920430A
:1008D0004F554E5420005B53455454494E47535D89
:1008E000002D204152445542554C4C4554202D007A
:1008F00000004D4152434820323032300050524FB8
:100900004752454D4D4544204259204F424F4E4F8E
:100910000000544849532050524F4752414D2049FE
:10092000530052454C454153454420554E44455291
:1009300000544845204D4954204C4943454E5345A9
:100940002E001B00080C0E0E0C0801030707030104
:1009500043414E43454C2020205354415254000003
:1009600000F8FFFFFF0FFFFFFFF0000000FFFFFF99
:10097000FFFF0F0FFFFFFFFEFC00FFFFFFFFFF0F5A
:100980000FFFFFFEFEFC00FFFFFFFFFF0000FFFF69
:10099000FFFFFF00FFFFFFFFFF0F0FFFFFFEFEF84F
:1009A00000FFFFFFFFFF0000FFFFFFFFFF00FFFF53
:1009B000FFFFFF00000000FFFFFFFFFF000000003F
:1009C000FFFFFFFFFF0F0F0F000F0F0FFFFFFFFFD6
:1009D000FF0F0F0FE0F0F8F8F83838F8F0F0E0808B
:1009E000FEFFFFFFE3E0E3FFFFFFFC8000FFFFFFF0
:1009F000FFFF0F0FFFFFFFFBF100FFFFFFFFFF00F7
:100A000000FFFFFFFFFF00FFFFFFFFFF0000FFFFF2
:100A1000FFFFFF00FFFFFFFFFF0F0FFFFFFDFDF8D0
:100A200000FFFFFFFFFF0000FFFFFFFFFF00FFFFD2
:100A3000FFFFFF00000000FFFFFFFFFF00000000BE
:100A4000FFFFFFFFFF0F0F0F00000000FFFFFFFF82
:100A5000FF000000878F9F9F3F7EFCFDF9F1E11FA3
:100A60001F1F1F1F0101011F1F1F1F1F001F1F1F0F
:100A70001F1F00001F1F1F1F1F001F1F1F1F1F1EE4
:100A80001E1F1F1F0F070003070F1F1F1E1E1F1F04
:100A90000F0F03001F1F1F1F1F1E1E1F1F1F0F07EB
:100AA0000003070F1F1F1E1E1F1F0F0F03001F1F16
:100AB0001F1F1F1E1E1E001F1F1F1F1F1E1E1E008A
:100AC0001F1F1F1F1F1E1E1E1E0000001F1F1F1F97
:100AD0001F000000070F0F1F1C1C1F1F0F0F070018
:100AE000000000003E5B4F5B3E3E6B4F6B3E1C3E8A
:100AF0007C3E1C183C7E3C181C577D571C1C5E7F9E
:100B00005E1C00183C1800FFE7C3E7FF001824181C
:100B100000FFE7DBE7FF30483A060E262979292651
:100B2000407F050507407F05253F5A3CE73C5A7F3B
:100B30003E1C1C08081C1C3E7F14227F22145F5F91
:100B4000005F5F06097F017F006689956A606060CB
:100B5000606094A2FFA29408047E040810207E2006
:100B60001008082A1C08081C2A08081E101010105B
:100B70000C1E0C1E0C30383E3830060E3E0E0600A1
:100B80000000000000005F00000007000700147F65
:100B9000147F14242A7F2A122313086462364956CC
:100BA00020500008070300001C2241000041221CC5
:100BB000002A1C7F1C2A08083E08080080703000AC
:100BC0000808080808000060600020100804023EC1
:100BD0005149453E00427F40007249494946214102
:100BE000494D331814127F1027454545393C4A4971
:100BF00049314121110907364949493646494929B0
:100C00001E000014000000403400000008142241BF
:100C10001414141414004122140802015909063E48
:100C2000415D594E7C1211127C7F494949363E4143
:100C30004141227F4141413E7F494949417F090964
:100C400009013E414151737F0808087F00417F41FF
:100C5000002040413F017F081422417F4040404036
:100C60007F021C027F7F0408107F3E4141413E7F8E
:100C7000090909063E4151215E7F09192946264985
:100C800049493203017F01033F4040403F1F20405C
:100C9000201F3F4038403F63140814630304780466
:100CA000036159494D43007F41414102040810202E
:100CB000004141417F0402010204404040404000A5
:100CC0000307080020545478407F284444383844AF
:100CD000444428384444287F385454541800087E2B
:100CE000090218A4A49C787F0804047800447D407D
:100CF000002040403D007F1028440000417F40001C
:100D00007C047804787C080404783844444438FC33
:100D10001824241818242418FC7C080404084854B7
:100D200054542404043F44243C4040207C1C204074
:100D3000201C3C4030403C44281028444C9090906B
:100D40007C4464544C4400083641000000770000A5
:100D5000004136080002010204023C2623263C1E04
:100D6000A1A161123A4040207A3854545559215576
:100D70005579412154547841215554784020545597
:100D800079400C1E527212395555555939545454E4
:100D90005939555454580000457C410002457D4264
:100DA0000001457C40F0292429F0F0282528F07C1A
:100DB000545545002054547C547C0A097F493249DB
:100DC0004949323248484832324A4848303A41412B
:100DD000217A3A42402078009DA0A07D39444444C5
:100DE000393D4040403D3C24FF2424487E49436631
:100DF0002B2FFC2F2BFF0929F620C0887E0903200A
:100E0000545479410000447D413048484A323840CA
:100E100040227A007A0A0A727D0D19317D2629292D
:100E20002F28262929292630484D4020380808082F
:100E30000808080808382F10C8ACBA2F102834FA50
:100E400000007B000008142A142222142A1408959A
:100E500000220095AA005500AAAA55AA55AA00008A
:100E600000FF00101010FF00141414FF001010FFFA
:100E700000FF1010F010F0141414FC001414F7000C
:100E8000FF0000FF00FF1414F404FC141417101FDB
:100E900010101F101F1414141F00101010F0000069
:100EA00000001F101010101F10101010F010000084
:100EB00000FF101010101010101010FF1000000094
:100EC000FF140000FF00FF00001F10170000FC04CB
:100ED000F414141710171414F404F40000FF00F7AE
:100EE00014141414141414F700F714141417141011
:100EF000101F101F141414F4141010F010F0000040
:100F00001F101F0000001F14000000FC140000F060
:100F100010F01010FF10FF141414FF141010101F05
:100F200000000000F010FFFFFFFFFFF0F0F0F0F016
:100F3000FFFFFF0000000000FFFF0F0F0F0F0F3833
:100F4000444438447C2A2A3E147E02020606027E6D
:100F5000027E0263554941633844443C04407E208C
:100F60001E2006027E020299A5E7A5991C2A492A9D
:100F70001C4C7201724C304A4D4D3030487848302C
:100F8000BC625A463D3E494949007E0101017E2A24
:100F90002A2A2A2A44445F444440514A4440404457
:100FA0004A51400000FF0103E080FF000008086B89
:100FB0006B083612362436060F090F060000181883
:100FC0000000001010003040FF0101001F01011E51
:100FD00000191D1712003C3C3C3C0000000000D5ED
:100FE000F08D1410A1C881CFD9F1AF20005D0E544F
:100FF0000E0619231D931C290EC81C44151E20081B
:101000000B000202020000090400000102020000BD
:101010000524001001052401010104240206052411
:101020000600010705810310004009040100020ABF
:10103000000000070502024000000705830240008F
:10104000000403090412010002EF020140412336AB
:101050008000010102030141726475696E6F204CCA
:101060004C430041726475626F790000482D112471
:101070001FBECFEFDAE0DEBFCDBF11E0A0E0B1E0F0
:10108000E8EAF8E602C005900D92A634B107D9F758
:1010900027E0A6E4B1E001C01D92AA3FB207E1F744
:1010A00018E0C7E3D8E004C02197FE010E9447344E
:1010B000C633D107C9F70E94832D0C9452340C9487
:1010C0000000EBE8F3E080E0A0E0B8E000800EBCB8
:1010D0008111012C1197A0FDFDCF0192B9F70DB43C
:1010E00008952091F80730E0209530954091F90758
:1010F00050E02423352390E02823392381E0232B5B
:1011000009F480E00895CF93DF93DC0177FF13C0EB
:1011100022273327261B370B842F042E000C990B14
:10112000281739072CF4460F70E060E0141644F0DD
:10113000DF91CF9108951416DCF760347105C4F780
:10114000A038B105A8F7262FCB01840F911D47FDCC
:101150009A958134910514F040E4461B27709FEF67
:10116000022E01C0990F0A94EAF7420F621B71091F
:1011700077FF02C0695F7F4F83E0759567958A9519
:10118000E1F7FB01F695FE2FEE27F795E795EA0FBD
:10119000FB1FE557FC4F28E030E06FEF70E01416BE
:1011A0003CF6483064F4D901A41BB10947FDB3955E
:1011B000EB0102C0D595C795AA95E2F79C238081E3
:1011C000982B90834850E058FF4F9FEFE8CF80E086
:1011D000EBE8F3E081118FEF0024819381938193F9
:1011E00081930394D1F7E1EEF7E0128A118A108A15
:1011F00017860895FC0180917203882311F13FB78F
:10120000F89482E08093E9002091F200822F90E030
:101210001816190614F481E090E0882339F0289814
:1012200044E6409371034091F1004083222339F05A
:101230002091F200211103C02BE62093E8003FBF6C
:1012400008958FEF9FEF08952FB7F89483E0809370
:10125000E9009091E800892F807295FF04C0909179
:10126000F20080E4891B2FBF0895809169038111EA
:101270000DC082E08093650384E080936603109242
:1012800068031092670381E08093690385E693E029
:101290000895CF93DF931F92CDB7DEB76983DC014A
:1012A000ED91FC910280F381E02D41E050E0BE0120
:1012B0006F5F7F4F09950F90DF91CF91089583E085
:1012C0008093E9008091F200882319F08AE38093EB
:1012D000E80008950E94240990E00895CF93DF93D9
:1012E0001F92CDB7DEB7FC018485958597FD08C0B8
:1012F0002FEF3FEF358724870F90DF91CF9108952F
:10130000CE0101960E94FA08019719F4898190E0B4
:10131000F3CF8FEF9FEFF0CF0F931F93CF93DF9318
:101320001F92CDB7DEB78C01FC018485958597FFB0
:101330000BC0CE0101960E94FA08019771F48981D1
:1013400090E0F80195878487F801848595850F9052
:10135000DF91CF911F910F9108958FEF9FEFF1CF04
:10136000FC018485958597FD0BC09FB7F89482E0BA
:101370008093E9008091F2009FBF90E0019608956C
:101380009FB7F89482E08093E9008091F2009FBFBC
:1013900090E0089540915F035091600320915D03B8
:1013A00030915E0342175307B4F49091E8009570B2
:1013B000E1F39091E80092FD19C08093F1008091D3
:1013C0005F039091600301968F739927892B19F41D
:1013D0008EEF8093E80080915F0390916003019607
:1013E0009093600380935F0381E0089580E0089507
:1013F000EF92FF920F931F93CF93DF93F82E192F45
:10140000E62E042F81E0860F880F0E94CA0983E030
:101410000E94CA09CF2DD12FEC0EFD2EF11CCE1546
:10142000DF05B9F007FF13C0FE0184910E94CA09CD
:10143000182F80E00E94CA09812321968111EFCFE5
:10144000DF91CF911F910F91FF90EF9008958881C8
:10145000EDCF81E0F5CFDF92EF92FF920F931F93D4
:10146000CF93DF93D82E8A01EB017B01E40EF51EAA
:10147000CE15DF0559F0D7FE12C0FE0184910E94FF
:10148000CA0921968111F4CF0FEF1FEFC801DF9138
:10149000CF911F910F91FF90EF90DF900895888179
:1014A000EECF0F931F93CF93DF931F92CDB7DEB78D
:1014B00082E0898342E450E06FEF7FE080E80E94A1
:1014C0002B0A0E943509DC0112960D911C91011521
:1014D000110589F0D801ED91FC910280F381E02D96
:1014E000BE016F5F7F4FC801099597FD04C0F801E9
:1014F00000851185ECCF89810F90DF91CF911F91ED
:101500000F910895615030F02091F100FC0120838B
:101510000196F8CF289884E6809371030895AF92DE
:10152000BF92CF92DF92EF92FF920F931F93CF93D0
:10153000DF936C017B018B01040F151FEB015E0132
:10154000AE18BF08C017D10759F06991D601ED91C7
:10155000FC910190F081E02DC6010995892B79F766
:10156000C501DF91CF911F910F91FF90EF90DF9018
:10157000CF90BF90AF9008953FB7F89480915403F7
:1015800090915503A0915603B091570326B5A89B9F
:1015900005C02F3F19F00196A11DB11D3FBFBA2F05
:1015A000A92F982F8827BC01CD01620F711D811DC5
:1015B000911D42E0660F771F881F991F4A95D1F74A
:1015C00008958F929F92AF92BF92CF92DF92EF9247
:1015D000FF926B017C010E94BC0A4B015C01C114AB
:1015E000D104E104F104B9F00E94BC0A6819790938
:1015F0008A099B09683E73408105910580F321E0CB
:10160000C21AD108E108F10888EE880E83E0981E1E
:10161000A11CB11CE4CFFF90EF90DF90CF90BF9062
:10162000AF909F908F9008958F929F92AF92BF92AC
:10163000CF92DF92EF92FF920F931F93CF93DF939E
:101640006C017B018A0180910F01882309F45CC041
:1016500080917203882309F457C08091640380FF4E
:1016600005C08091E00082608093E000E801B12C29
:101670008AEFA82E93E0892E2AE3922E209711F468
:10168000BB20D9F10E94240981110AC0AA94AA2082
:10169000D9F161E070E080E090E00E94E10AEECFD5
:1016A0008C171D0611F00CF08C2F9FB7F8948092C8
:1016B000E9002091E80025FD02C09FBFDFCF282F61
:1016C00030E0C21BD30BF701815020F041914093D1
:1016D000F100FACFE20EF31EBB2021F09092E80059
:1016E000B12CEBCF8091E80085FDE7CF9092E80028
:1016F000BB24B394209709F3F3CF5D9884E68093DD
:101700006303101611063CF081E090E0F60193832C
:10171000828310E000E0C801DF91CF911F910F910B
:10172000FF90EF90DF90CF90BF90AF909F908F9001
:101730000895BC0190E080E00C94E10A8FB180959F
:10174000807F669B88601C9B846008958091520313
:101750000895109252033E983F9808953E9A3F9AFA
:1017600081E08093520308953F924F925F926F926F
:101770007F928F929F92AF92BF92CF92DF92EF9221
:10178000FF920F931F93CF93DF9330E0F901E80F9F
:10179000F91FF7FDD5C0803891050CF0D1C0FB01D1
:1017A000E00FF11DF7FDCCC0603471050CF0C8C02E
:1017B000DB0177FF04C0AA27BB27A61BB70BA770C6
:1017C000BB27FB0177FD3796C3E0F595E795CA95F2
:1017D000E1F777FF07C0319768E070E0EB01CA1BC3
:1017E000DB0BDE01402E469446944694512C077044
:1017F00019F0DFEF4D1A5D0ABF01EF01D695DC2F1E
:10180000CC27D795C795C80FD91FC557DC4F8A017C
:10181000460E571E48E050E04A018A1A9B0A64159A
:10182000750509F48DC06830710509F489C06F3FF2
:10183000EFEF7E070CF44BC06C0150E040E03E013E
:10184000E0E86E0E711CD7FC35C06F3F760709F4D7
:1018500073C05E01A40EB51EF501F080FA01E00F21
:10186000F11F33243394E31039C0E4910A2E01C0F0
:10187000EE0F0A94EAF7FE2AF501F0821097D1F0F4
:1018800067307105B9F05301A40EB51EF501F08063
:10189000FA01E00FF11F33243394E31035C0E491D3
:1018A000F0E0082C02C0F595E7950A94E2F7FE2ACD
:1018B000F501F0824F5F5F4FFFEFCF1ADF0A42174B
:1018C00053072CF4F0E8CF16D10409F0BCCF6F5FBA
:1018D0007F4FC058DF4F020F131FA1CFE1100CC084
:1018E000E491F0E00A2E02C0EE0FFF1F0A94E2F727
:1018F000E095F095FE22C0CFE4910A2E01C0EE0FD4
:101900000A94EAF7FE26B8CFE1100CC0E491F0E0AB
:10191000082C02C0F595E7950A94E2F7E095F0955A
:10192000FE22C6CFE491F0E0082C02C0F595E795C1
:101930000A94E2F7FE26BCCF109709F0A4CFBACFE5
:10194000DF91CF911F910F91FF90EF90DF90CF909B
:10195000BF90AF909F908F907F906F905F904F90CF
:101960003F9008956F927F928F929F92AF92BF9215
:10197000CF92DF92EF920F931F93CF93DF936C017F
:101980005B014A01122FC1E0D0E083E0682E712C88
:10199000CE01B3010E9433346A0D7B1D6150710981
:1019A0008C0D9D1DE12C00E1212FA40101970E94C7
:1019B000B40B2296C930D10559F7EE24E394212FB8
:1019C000A401B501C6010E94B40BDF91CF911F9114
:1019D0000F91EF90DF90CF90BF90AF909F908F903E
:1019E0007F906F90089580389105B8F46034710548
:1019F000A0F420E191E061FD94E060FD990F62FDAB
:101A00009295687F269FD0011124A80FA557BC4F3F
:101A10008C9140FF03C0892B8C9308959095892366
:101A2000FBCF2F923F924F925F926F927F928F9255
:101A30009F92AF92BF92CF92DF92EF92FF920F935D
:101A40001F93CF93DF93CDB7DEB72A970FB6F894E5
:101A5000DEBF0FBECDBF9A8389836A3061F5DC019A
:101A600055968C91B8E08B9F90011124E981FA8101
:101A700081899289820F931F928B818B108A17869E
:101A800081E090E02A960FB6F894DEBF0FBECDBF7E
:101A9000DF91CF911F910F91FF90EF90DF90CF904A
:101AA000BF90AF909F908F907F906F905F904F907E
:101AB0003F902F9008956D3019F329813A813A872C
:101AC0002987D9011F96AD90BC90B0E8AB16B10440
:101AD0000CF07BC0F901C188D288F0E4CF16D104A4
:101AE0000CF073C0D90155966C90559745E095015F
:101AF000649E200D311D1124121613060CF065C0D2
:101B0000262C312C910153E0220F331F5A95E1F717
:101B10002C0D3D1D121613060CF057C05496BC91A7
:101B2000BB83E985FA85F389FC83649FB0011124A6
:101B30009B012152354F3A832983712CE981FA8127
:101B40008491F5E07F1201C080E0460138E0532E19
:101B5000282F30E03E832D834C8080FF4B80411046
:101B600004C03B818C813817E1F010E000E00615DD
:101B7000C0F4D501A00FB11FB887AF83F12CE12CC1
:101B8000E61460F4B701680D791D442D8F819885A6
:101B90000E94F30CBFEFEB1AFB0AF2CF0F5F1F4F4F
:101BA000E6CF8D819E81959587955A94820C931CE2
:101BB0005110CECF7394E981FA813196FA83E9838B
:101BC000A20CB31CF6E07F12B9CFA985BA85559651
:101BD0002C915597422F50E01F968D919C91B6E025
:101BE0002B9F800D911D1124E985FA85908B8787A5
:101BF0002689222309F444CF6AEF64039001659F8C
:101C0000300D112420583F4F281739070CF038CFDA
:101C1000DF010190F081E02D0190F081E02D6AE07C
:101C2000CD0109952DCF0895EF920F93EE24E39403
:101C300005E120E84FE559E068E070E090E080E0E1
:101C40000E94B40B0F91EF90089585E080933E03BE
:101C50000895CF93C0913E03C53089F08091510320
:101C600081110E94E708EC2FF0E0EE0FFF1FE9560C
:101C7000F84F85919491FC01099510925103CF91F1
:101C800008959C019091360396306CF484E098029C
:101C9000F0011124EF5EFC4F338322837183608354
:101CA0009F5F90933603089590914B0391509093CA
:101CB0004B0381E0911180E0089588E780934B0306
:101CC00008959091C901903419F1A0910201B09149
:101CD0000301FD0130813F7141F03596AAECB1E07E
:101CE00033E0EA30F307B0F3F4CFF0930301E0936D
:101CF000020182836383448312165CF420320CF069
:101D00002FE12F712F71208311829F5F9093C90162
:101D1000089521E0F7CF8F929F92AF92BF92CF921A
:101D2000DF92EF920F931F93CF93DF936C015B01D0
:101D3000C42FD22F802E912C023070F094012150AC
:101D400031094E2D4203C001439F900D112497FD90
:101D5000019695958795C81B10E000E008151905B8
:101D600054F42D2F4C2FB501C6010E94610E0F5F58
:101D70001F4FCE0DF3CFDF91CF911F910F91EF90B9
:101D8000DF90CF90BF90AF909F908F900895E4E543
:101D9000F1E0808187FD02C08B5F8083329681E015
:101DA000E837F807B1F708959091F90796FB3327C4
:101DB00030F995FB882780F9381B94FB552750F99B
:101DC000892F881F8827881F581B8091510142E066
:101DD000883031F0332319F043E0511101C044E061
:101DE00020910C03349F200D1124243FD8F023EFC1
:101DF00020930C0330910B03549F300D1124343F7A
:101E0000A8F033EF30930B0392FF45C0909150013F
:101E1000911103C09CE090935001883058F080915C
:101E200050010FC02C3020F72CE0E2CF3C3050F7AF
:101E30003CE0E8CF8F5F809351018091500188236F
:101E4000A9F14FEF480F4093500163E00E94133413
:101E500091112CC08BEA489F412D1124469584E0B6
:101E6000841B269526952B5F36953695E0910001CB
:101E7000F09101012083932F981B91832283380FC7
:101E80003383349681E0E837F80748F4F093010192
:101E9000E09300010895882381F28150CCCF84E53E
:101EA00091E0909301018093000108950895282FF7
:101EB0008091430385FF1DC0E22FF0E0E956FA4F01
:101EC000E4918E2F69E10E94133480934F0135E035
:101ED0008E2F632F0E941334492F0E941334909346
:101EE0004E0140934D0188E0253009F480E1809354
:101EF0004C010895E82F87FF04C071956195710921
:101F0000EF77E1341CF080E88E1BE82F0E2E000CDA
:101F1000FF0BE454FD4FE491E69FC001E79F900D55
:101F20001124880F892F881F990B0895CF92DF9273
:101F3000EF92FF920F931F93CF93DF93EC01888171
:101F4000282F2295269527709981892F880F880F31
:101F5000880F822B9295969597706CE070E00E94A6
:101F600033346B010B8110E08C810E947A0F080FD3
:101F7000191FEA80F12C8C81B601805C0E947A0FD7
:101F8000A701480F591FC801BA01DF91CF911F91D6
:101F90000F91FF90EF90DF90CF9008959F92AF92B6
:101FA000BF92CF92DF92EF92FF920F931F93CF9346
:101FB000DF9300910B030695069510E0780181E010
:101FC000E81AF108C0910C03C695C695D0E06E01E1
:101FD000E1E0CE1AD1088AECA82E81E0B82E912C2F
:101FE00022960E5F1F4FF5013081232F2F7109F4C8
:101FF00042C03295369537704181542F550F550F99
:10200000550F852F832B942F929596959770820F5D
:10201000911D382F3295330F307E232B20839295DC
:10202000990F907E869586958695892B8183C5012B
:102030000E94960F9B014091DB075091DC076417CB
:1020400075077CF1E091DF074E0F511D641775078E
:1020500044F56091DD077091DE07861797070CF154
:102060004091E007460F572F511D84179507CCF478
:102070002C153D0504F5F5E0AF0EB11C8AE0A8165D
:1020800083E0B80609F0AFCF892DDF91CF911F9182
:102090000F91FF90EF90DF90CF90BF90AF909F9007
:1020A0000895F5018081807E80838091C9018150EF
:1020B0008093C901E0CF2C173D07ECF68E159F05E4
:1020C000D4F280179107BCF699249394D4CFCF9281
:1020D000DF92EF92FF920F931F93CF93DF937C01D8
:1020E0008B01DB011296EC91E40FF52FF11DDC0161
:1020F0001296CC9012978C2D8F738E9F90018F9F8C
:10210000300D11246C91962F92959F7011964C91E1
:10211000642F63706295607F692B70E0C9010E9433
:102120001F34D62E242F269526952F71D801CC91B9
:102130008C2F82958695869583701196CC91CF7061
:10214000CC0FCC0FC82BD0E030E0C294C694C6941C
:1021500083E0C822D70113969C919F70990F990F25
:102160009C299E9FB0019F9F700D1124CB01B90146
:102170000E941F34862F4078B901840F0E947A0F85
:10218000C80FD91FF80100810F7310E0005C1F4FCA
:10219000D7016C91862F82958F7011966C91637028
:1021A0006295607F682B70E080E48D0D0E947A0F4D
:1021B000A801480F591FCE01BA01DF91CF911F919D
:1021C0000F91FF90EF90DF90CF900895EF920F93D3
:1021D00027E0429FA001112442555D4FE090F40793
:1021E00007E027E00E94B40B0F91EF900895109242
:1021F0003503109234038091F907982F907F41F1B5
:1022000090914A019F5F94310CF590934A0190910F
:102210004A01913011F09F30E9F485FF03C09FEF30
:102220009093340386FF05C0909134039F5F909391
:10223000340387FF03C09FEF9093350384FF0AC0E8
:10224000809135038F5F8093350308959FE0DDCF44
:1022500010924A010895E0E4F3E02081318145E0E5
:10226000429FC001439F900D11244281538167E03A
:10227000649F9001659F300D1124820F931F875C2E
:1022800093484481558169E0649F9001659F300DBA
:102290001124280F391F468157816BE0649FC001CC
:1022A000659F900D1124820F931F408551856DE02D
:1022B000649F9001659F300D1124820F931F089534
:1022C000CF92DF92EF92FF920F931F93CF93DF9302
:1022D000082F142F469FE001479FD00D1124F12CA9
:1022E000E12C60E074E284EF90E0A7019E010E947F
:1022F000A030215031094109510991E021153105E2
:1023000081E0480751056CF060E970ED83E090E0F2
:10231000A7019E010E94A0302150310941095109B5
:1023200093E0013059F00330F9F0DF91CF911F9124
:102330000F91FF90EF90DF90CF9008951093480198
:1023400080918100887F892B809381003093890060
:1023500020938800109285001092840080916F0075
:10236000826080936F00E1CF10934901D0934701C1
:10237000C093460180919100887F892B80939100C2
:102380003093990020939800109295001092940039
:1023900080917100826080937100C7CF811116C057
:1023A0001092840380917A0381110AC080912C03DA
:1023B000E0912D03F0912E039081809589238083F5
:1023C00042E064EF71E083E00C94601180917F0340
:1023D000811110C080916F008D7F80936F0080917C
:1023E0002903E0912A03F0912B03908180958923A2
:1023F000808308950895FF920F931F93CF93DF93E7
:10240000EC0190918A03992309F464C08B01913007
:1024100071F480918903882351F0809188038F3F64
:1024200009F058C080E00E94CE1110928903E0911B
:102430008603F09187030995FF24F3948F258093F9
:10244000850330E020E0A9019801220F331F441FCB
:10245000551FDE010E94BF306C507E4F8F4F9F4F43
:1024600028EE33E040E050E00E94D23080918A03B1
:102470008130A1F4809384032093800330938103FF
:10248000409382035093830383E042E0BE01DF91D7
:10249000CF911F910F91FF900C946011F0927F03E8
:1024A00020937B0330937C0340937D0350937E0302
:1024B00080918903882351F081E0909188039F3FA8
:1024C00009F080E080937A0381E0DFCF8FEF809383
:1024D0008803FACFDF91CF911F910F91FF9008955C
:1024E00064E170E08BE492E00C94FB110E947012A6
:1024F000E0E4F3E020913F032D5F81E090E0A0E075
:10250000B0E004C0880F991FAA1FBB1F2A95D2F7FD
:1025100023818227838381E08093500308950E9462
:102520007012E3E4F3E02081822F8F7090E06AE084
:1025300070E00E9433348F5F8F70207F282B2083C0
:1025400081E08093500308950E94701283E080938D
:102550003E0381E08093510308950E94701210920F
:1025600036036FE872E185EE97E00E94410E66E760
:1025700072E18DED97E00E94410E66E772E183ED16
:1025800097E00E94410E66E772E187EC97E00E94B7
:10259000410E6BEE72E182EC97E00E94410E1092C8
:1025A0003F0381E08093370392E090933D032CE05A
:1025B00020933C032CE720933B032EE120933A0326
:1025C000109239031092380390933E038093510385
:1025D00080935003089580913E03823011F40E944D
:1025E0007012109236038091480390914903892B11
:1025F00061F065E27EE08CEB97E00E94410E70E0B6
:1026000060E090E080E00E94410E6EE07CE181EBB2
:1026100097E00E94410E6DEA72E188EA97E00E941D
:10262000410E64EA72E181EA97E00E94410E8091D6
:102630003E038230E9F480913603825080933F0359
:1026400081E0809337039CE290933D0396E2909360
:102650003C0394E590933B039AE190933A031092E4
:1026600039038093380380933E0380935103089588
:102670008091430387FB882780F9880FDFCF8CE0A8
:102680000E947108882339F00E94701281E08093C3
:102690003E038093510308950E94701210920A0322
:1026A00081E0809351030895CF93DF93C0913F035E
:1026B00086E0C802E0011124A6960E9470121092D2
:1026C000360361E178E28AEB95E00E94410E6CE40A
:1026D00073E183EB95E00E94410E88E280933D0315
:1026E000C0933C038FE280933B038BE080933A03DB
:1026F00081E0809339038093380380933F03809374
:102700003703DF91CF910895CF930E9470121092FA
:102710003603C0910F03C230B8F161E27DE188E871
:1027200095E00E94410E64E573E1C13011F061E172
:1027300078E28AE795E00E94410E90913603892F56
:10274000880F890F880F93E190933D0396E3981BC0
:1027500090933C0399E590933B03815080933A0317
:1027600091E0909339039093380380914B0189272E
:10277000C23009F080E080933F0381E0809337030B
:1027800080930A03CF9108956CE473E18EE895E09D
:102790000E94410ECC2359F2C0CF6AE070E088EB72
:1027A00091E00C94FB118F929F92AF92BF92CF92C7
:1027B000DF92EF92FF92CF93DF9380E40E94710843
:1027C000F82E80E20E947108F81AC1F080914A0345
:1027D0002F2D0F2C000C330B820F932F911D8F3F49
:1027E000980761F0059754F40E94CD1380914A0335
:1027F000F80EF0924A0381E08093500380913503F4
:10280000882309F457C00E94CD13C0914A03D0E039
:10281000F0E0E0E0C12CD12C7601C394EC17FD0769
:1028200054F43196ABE1B0E0A70196010E94BF30AD
:102830006B017C01F3CF80904C0390904D03A090EE
:102840004E03B0904F03C0913503C501B401A701F9
:1028500096010E94A030CA01B9012BE130E040E0AE
:1028600050E00E94A0302C2F0C2E000C330BC9011D
:10287000860F971F4B9740F0A6EEBFEFA70196017A
:102880000E94CD306B017C01AC2FCC0FBB0BA7019C
:1028900096010E94CA30860E971EA81EB91E80920D
:1028A0004C0390924D03A0924E03B0924F0381E0EF
:1028B0008093500388E00E947108882391F00E9461
:1028C000701281E080933E0380935103DF91CF919A
:1028D000FF90EF90DF90CF90BF90AF909F908F9040
:1028E000089584E00E947108882381F340914C038D
:1028F00050914D0360914E0370914F0380914003BE
:1029000090914103A0914203B0E084179507A60778
:10291000B70729F0809143038F7780934303409357
:102920004003509341036093420385E080933E034C
:10293000CDCF80E80E9471088823C1F080913F03C9
:102940001816A4F48150982F815024E09202F001CF
:102950001124EF5EFC4F20813181232BA1F3909352
:102960003F030E94CD1381E08093370380E10E94F2
:102970007108882321F180913F03482F082E000C15
:10298000550B20913603022E000C330B21503109D8
:1029900042175307A4F48F5F982F8F5F24E09202B1
:1029A000F0011124EF5EFC4F20813181232BA1F334
:1029B00090933F030E94CD1381E080933703809171
:1029C0003803882381F088E00E947108882359F039
:1029D00080915203811118C00E94AE0B0E947012A8
:1029E00081E08093370384E00E947108882379F0A6
:1029F000E0913F0384E0E802F0011124EF5EFC4F18
:102A00000190F081E02D09940E94A90BE7CF089571
:102A100080913F03882379F087FD02C0843064F100
:102A20000E94991480E90E947108882319F081E0BE
:102A300080935003089580913403882389F30E9482
:102A4000CD1320914303822F8F708150990B3091C9
:102A50003403830F911D37FD9A950A966AE070E062
:102A60000E9433348F5F8F70207F282B2093430385
:102A700081E080935003D4CF80E60E9471088823C0
:102A800079F20E947612CCCF0E94F71080910A034F
:102A9000882341F00E94991480910F038330D1F074
:102AA00082E0089580914B038F5F80934B03809168
:102AB0004C01882319F0815080934C01E0910F0361
:102AC000F0E0EE0FFF1FED5EFC4F85919491FC014D
:102AD0000995E2CF81E00895FF920F931F93CF9362
:102AE000DF9301E010E0FF24F394E0917603F0918E
:102AF0007703AF014F5F5F4F5093770340937603A7
:102B00002491822F807FC22FCF70D22FD370803834
:102B100021F48D2F0E94CE11E8CF803909F03FC0FB
:102B2000E0918603F091870309958F2580938503B3
:102B3000E0917603F0917703CF01019690937703AC
:102B400080937603E4918091750390918A03D9175D
:102B500060F6D13021F490917F039111C6CF8E0F92
:102B600087FDC3CFE82FF0E08C3390F4EE59FD4F92
:102B7000E4916E2F70E081E0D11103C0F0928403E4
:102B800083E04C2F469546954E5F0E946011ADCF75
:102B9000EE0FFF1FEE59FE4F65917491ECCF87FD4C
:102BA0003FC03296F0937703E0937603FA014491A5
:102BB000A0914601B0914701322F242F0E94F4309A
:102BC0006C507E4F8F4F9F4F28EE33E040E050E037
:102BD0000E94D2302093800330938103409382037C
:102BE000509383038091800390918103A09182038D
:102BF000B0918303892B8A2B8B2B61F481E090E0C9
:102C0000A0E0B0E08093800390938103A0938203BF
:102C1000B0938303DF91CF911F910F91FF9008959F
:102C2000803DA1F4F0937903E093780380917303DE
:102C3000882309F45ACFEC2FF0E0E256FD4FE491DF
:102C4000C0917503EC0FE09375034FCF803E21F5E3
:102C5000C11109C080917803909179039093770313
:102C60008093760342CF809173038F5F80937303C9
:102C7000980102C0220F331FCA95E2F7821713068C
:102C80004CF35093790340937803809174038093BD
:102C900075031092730329CF803F09F026CF10925D
:102CA0008903B8CF0F931F93CF93DF938C01D62F57
:102CB00080918903882349F180918803861790F1D8
:102CC000C0E080918A03C81728F48C2F0E94CE118F
:102CD000CF5FF7CF10928903D093880310937903C5
:102CE0000093780310937703009376031092750393
:102CF000109274031092730381E080938903DF9133
:102D0000CF911F910F910C946C1580917F038823B4
:102D100019F381E090918803961708F080E0809382
:102D20007A03DACFDF91CF911F910F910895EF923F
:102D30000F93CF93DF9377FF0CC088279927861BCB
:102D4000970B2817190609F00CF47CC0260F70E0C9
:102D500060E057FF0FC0EE27FF27E41BF50B802F25
:102D6000002E000C990BE817F9070CF06BC0040F4C
:102D700050E040E0222309F465C0603871050CF092
:102D800061C010160CF05EC0403451050CF05AC002
:102D9000CB01820F911D8138910514F020E8261B8C
:102DA000942FFA01E00FF11D07FDFA95E134F105CA
:102DB00014F000E4041B97708FEF092E01C0880FF8
:102DC0000A94EAF7090F491B510957FF02C0495FEE
:102DD0005F4F93E0559547959A95E1F75695542F97
:102DE000442757954795640F751F65577C4F48E0FA
:102DF00050E0AFEFB0E010162CF5083064F4FA01A3
:102E0000E01BF10907FDF395ED0102C0D595C795CB
:102E1000EA95E2F78C23E1100DC08095FB01922F1B
:102E20003081382331939150D9F7085060587F4F43
:102E30008FEFE1CFFB01922F3081382B31939150EE
:102E4000D9F7F3CFDF91CF910F91EF9008952F92A3
:102E50003F924F925F926F927F928F929F92AF922A
:102E6000BF92CF92DF92EF92FF920F931F93CF9377
:102E7000DF9300D000D01F92CDB7DEB79B838A834B
:102E80006A3061F5DC0155962C91559751968D91DC
:102E90009C91B6E02B9F800D911D1124EA81FB814E
:102EA000928B818B108A178681E090E00F900F90B3
:102EB0000F900F900F90DF91CF911F910F91FF9086
:102EC000EF90DF90CF90BF90AF909F908F907F90CA
:102ED0006F905F904F903F902F90089580EE860FF7
:102EE000803410F72A813B813D832C83D9011F96C2
:102EF000CD90DC90B0E8CB16D1040CF048C0F901BD
:102F0000A188B288F0E4AF16B1040CF040C0D9013A
:102F100055961C91C601B5E01B9F800D911D112493
:102F200097FD35C0C501E6E01E9F800D911D11245F
:102F300097FD2DC0D9015496FC90549753962C9030
:102F4000B4E06B9FF0011124E65AFF4F4590559075
:102F500065907490113009F050C0460116E0D12CF4
:102F6000C12C40FC42C04F2DF21040C076946794B3
:102F700057944794EFEFCE1ADE0AF6E0CF16D1044D
:102F800081F711502FEF821A920A1111E8CFAC810C
:102F9000BD8155962C915597422F50E01F968D91EB
:102FA0009C91B6E02B9F800D911D1124EC81FD8139
:102FB000908B87872689222309F476CF6AEF6403F2
:102FC0009001659F300D112420583F4F2817390775
:102FD0000CF06ACFDF010190F081E02D0190F081CB
:102FE000E02D6AE0CD0109955FCF422DB5016C0D52
:102FF0007D1DC4010E94F30CB9CF812F90E09B830B
:103000008A8396E09983450196E0392E40FC18C0EA
:10301000EF2CF21016C076946794579447943A9424
:10302000AA81BB818A0E9B1E3110F0CFB981B150AD
:10303000B983EA81FB81CE0EDF1EB111E4CFA7CFA9
:10304000E22C012F212FA401B6018C819D810E94C9
:103050009716E1CF0C9427178F929F92AF92BF9251
:10306000CF92DF92EF92FF92CF93DF9369017A01C3
:103070009093F1078093F0077093F3076093F20742
:10308000C5E0D0E08BE1882E912CA12CB12CC7019A
:10309000B601A50194010E94D2306A317105D1F0C8
:1030A0006F5B81EE97E00E942A18C701B601A50167
:1030B00094010E94D23069017A01219741F7DF9192
:1030C000CF91FF90EF90DF90CF90BF90AF909F9007
:1030D0008F9008956EE2E5CF0F931F93CF93DF9308
:1030E0008C01D0E0C0E0F801EC0FFD1F6491662375
:1030F00041F081EE97E00E942717892B11F021966D
:10310000F2CFCE01DF91CF911F910F910895CF9211
:10311000DF92EF920F93CF9380915103882301F1B7
:103120000E94140E8CE190E09093F1078093F007D9
:1031300089E390E09093F3078093F20780E599E0AC
:103140000E946C1840E068E370E080E190E00E942B
:10315000E61041E068E370E086E490E00E94E6104B
:1031600080915003882319F18091510381110BC084
:10317000E12C02E126E341E250E065E270E081EEFD
:1031800097E00E94971682E08093F60720914C0307
:1031900030914D0340914E0350914F0365E270E032
:1031A00083E290E00E942C1881E08093F607C091A2
:1031B0004B0380915003811103C08C2F8370F1F475
:1031C000C2FBCC27C0F9C0904A038CE0C89E6001C6
:1031D000112485E2C80ED11CEC2E03E026E044E465
:1031E00059E060E270E0C6010E94B40B26E04AE4B8
:1031F00059E060E370E0C6010E94B40B10925003E6
:10320000CF910F91EF90DF90CF9008956F927F92C2
:103210008F929F92AF92BF92CF92DF92EF920F93D5
:10322000CF93DF9380914B038F50990B63E070E055
:103230000E9433348AE39AEAA3EEBEEE04C0B69548
:10324000A795979587956A95D2F7C82FC1708FE794
:10325000C89F802D112493E894BD9FEF97BD91EFF7
:10326000909380008093880010928A000E94E70863
:1032700020914B0388E790E0821B91096CE270E09B
:103280000E9433343B0187EFA82E85E0B82E9CE1E5
:10329000892E912CD12CC12CD0E081E090E06C14CF
:1032A0007D0411F090E080E08C9FB0018D9F700D47
:1032B0009C9F700D1124645F7F4FEE24E39400E225
:1032C00028E1A501C4010E94B40B8FEFC81AD80AE7
:1032D00088E1880E911C80E6A80EB11C83E0C81618
:1032E000D104D9F608E020E247ED55E06CE270E049
:1032F00084E490E00E94B40B80E190E09093F107A9
:103300008093F0078AE390E09093F3078093F207AD
:1033100086EC95E0DF91CF910F91EF90DF90CF9009
:10332000BF90AF909F908F907F906F900C946C188F
:10333000089590E080E0089597FF0DC0222733277D
:10334000281B390B4217130629F024F0480F90E090
:1033500080E031F408954423E9F380389105D4F7EF
:1033600060347105B8F79C01240F311D21383105F7
:1033700014F040E8481B362F377021E001C0220FBF
:103380003A95EAF7FB0133E0F595E7953A95E1F7D1
:10339000F695FE2FEE27F795E795E80FF91FE5570D
:1033A000FC4F8081822B81934150D9F7D3CFBF92BC
:1033B000CF92DF92EF92FF920F931F93CF93DF9301
:1033C000C0904B03CC2DC37087E4C89FD02C112430
:1033D00083E0C89F800111240952164EB0900F035C
:1033E000E0900D03F0900E03B11004C0EC2DE857EF
:1033F000FF0B7F01D0E0CC0FDD1FF8018491835ECD
:10340000D80E3196E4918D2D90E0EF70F0E0389673
:10341000EE9D9001EF9D300DFE9D300D112446E094
:10342000359527954A95E1F7821B930B41E0BE0144
:103430008F7799270E94F30C2896045F1F4FC034A2
:10344000D105DCF28091430386FF31C0F1E0FB152A
:1034500070F1C0FC2CC0C0910C03C695C695CB5032
:10346000DD0B10910B03169516951C161D064CF0DE
:1034700047E1812F8B50990BBC0190E080E00E94C6
:10348000830847E170E060E01C3028F0143378F0E6
:1034900047E16FE370E0CE01DF91CF911F910F9173
:1034A000FF90EF90DF90CF90BF900C949C19DF912C
:1034B000CF911F910F91FF90EF90DF90CF90BF9031
:1034C00008958F929F92AF92BF92EF92FF920F93C7
:1034D0001F93CF93DF93CDB7DEB7A1970FB6F894C4
:1034E000DEBF0FBECDBF7C01FA01CB0119A2223095
:1034F00008F42AE08E010F5D1F4F822E912CB12C13
:10350000A12CBF01A50194010E94D230F901CA018A
:103510006A304CF5605DD8016E938D01232B242B0E
:10352000252B79F790E080E0109761F0FD01019084
:103530000020E9F73197AF014A1B5B0BBD01C701C2
:103540000E948F0AA1960FB6F894DEBF0FBECDBFC2
:10355000DF91CF911F910F91FF90EF90BF90AF90AF
:103560009F908F900895695CD6CFEF920F93CF9381
:10357000DF9381E0909110039A3008F480E0C82F27
:10358000D0E09E01220F331F220F331FC21BD30B2B
:10359000282F220F280F220F255ABE016E5E7F4F63
:1035A000E12C07E040E150E081EE97E00E949716A1
:1035B000CE0143969093F1078093F00781E190E06C
:1035C0009093F3078093F2078DEB95E00E946C18BF
:1035D00020914003309141034091420350E061E16A
:1035E00070E0CE018D5B9F4F0E942C186DE281EE42
:1035F00097E00E942A184091100350E070E060E0CC
:103600002AE081EE97E0DF91CF910F91EF900C943B
:10361000611A2F923F924F925F926F927F928F9298
:103620009F92AF92BF92CF92DF92EF92FF920F9351
:103630001F93CF93DF939093F1078093F0077093DC
:10364000F3076093F20769017A01CA01B90120EC1E
:103650003BE443E050E00E94D23029013A01C70127
:10366000B60120E13EE040E050E00E94D2308CE321
:10367000882E912CA12CB12CCA01B901A50194016D
:103680000E94D230D62F272E382E092FC701B6011F
:10369000A50194010E94D230CA01B901A50194018B
:1036A0000E94D230C62F972E5C018C2E41145104FB
:1036B00009F03FC0D11150C06A3028F460E381EEB8
:1036C00097E00E942A182AE04C2F592DB50181EE6F
:1036D00097E00E94611A6EE281EE97E00E942A183C
:1036E000C701B60126E030E040E050E00E94D23051
:1036F000CA01B9012AE030E040E050E00E94D23037
:10370000AB01BC012AE081EE97E0DF91CF911F91E0
:103710000F91FF90EF90DF90CF90BF90AF909F9070
:103720008F907F906F905F904F903F902F900C9470
:10373000611A2AE0B301A20181EE97E00E94611AAA
:103740006AE381EE97E00E942A18DA3028F460E3F9
:1037500081EE97E00E942A182AE04D2F522D632D0A
:10376000702F81EE97E00E94611A6AE381EE97E084
:103770000E942A1829E0281528F060E381EE97E0DE
:103780000E942A182AE04C2F592DB501BCCF0E9467
:103790004D34CF92DF92EF92FF920F931F93CF930E
:1037A000DF9380915103882381F10BE010E0C1EE9B
:1037B000D8E0FE0184918B3141F165E170E0CE01EA
:1037C0000E944C307C016C01DD24282F3DEF320338
:1037D000C0011124805C9F4F9093F1078093F00704
:1037E0001093F3070093F207CE010E946C188FEF3D
:1037F000C81AD80ACC0DDD1D86E090E0E11002C0A9
:1038000082E090E0080F191FD4CFDF91CF911F9174
:103810000F91FF90EF90DF90CF9008958F929F923D
:10382000AF92BF92CF92DF92EF92FF92CF93DF934E
:103830008091430384FF4CC00E94701210924A038F
:103840008091400390914103A0914203B0E08B36F8
:1038500022EF92072AEDA20701F5C5E0D0E020E0B3
:1038600030E0A9019AE1C92ED12CE12CF12CABE179
:10387000B0E00E94BF304B015C010E94EB2FA7011A
:1038800096010E94A0309B01AC01280D391D4A1DF4
:103890005B1D219761F7DA01C90180934C03909376
:1038A0004D03A0934E03B0934F0384E080933E03F7
:1038B00081E08093510380935003DF91CF91FF907B
:1038C000EF90DF90CF90BF90AF909F908F90089532
:1038D0008F7780934303C5E0D0E020E030E0A9017A
:1038E0008AE1C82ED12CE12CF12CABE1B0E00E9492
:1038F000BF304B015C010E94EB2FA70196010E9493
:10390000A0309B01AC01280D391D4A1D5B1D21977C
:1039100061F720934003309341034093420385E0D5
:1039200080933E03CACFCF92DF92EF92FF920E9424
:10393000F71080914B038F5F80934B03E0913E0320
:10394000F0E0EE0FFF1FE357F84F85919491FC01D3
:1039500009950E948F2F6C01990FEE08FF080E94B5
:10396000BC0AC616D706E806F90631F06C257D2597
:103970008E259F250E943A3080913E03853031F09C
:1039800081E0FF90EF90DF90CF90089582E0F9CF33
:1039900060E08DEF92E00E945216809143038F7099
:1039A0008093100310920E0310920D0380E4809315
:1039B0000C0380E880930B03109250011092510188
:1039C00010924B01E4E5F1E08083329691E0E83714
:1039D000F907D1F7EAECF1E08081807E80833596AB
:1039E00083E0EA30F807C1F71092C901E8E7F1E097
:1039F00081818F708183349691E0E43BF907C1F7B0
:103A0000809153018F71806C8093530180914003AA
:103A100090914103A0914203B0E0BC01CD016F5FE2
:103A20007F4F8F4F9F4F0E943A3010924B0310925E
:103A30004C0110920A0310920F0381E0809351030E
:103A400008950C94C81C0F931F93CF93DF9380911C
:103A50003E038111B4C086EA9BE090938703809374
:103A6000860380918A038823B1F190E023E080915E
:103A70008A03981750F5911116C0809171008D7FBF
:103A80008093710080912C03E0912D03F0912E031F
:103A90003081809583238083809165008860809346
:103AA00065009F5FE4CF80916F008D7F80936F00F2
:103AB00080912903E0912A03F0912B0330818095B6
:103AC0008323808320938100ECCF10927A0310929D
:103AD0007F031092890381E080938A03E3E7F7E094
:103AE0008491E4E5F7E0249190E0880F991FFC01B0
:103AF000EF5BF84F45915491FC01ED5CF84FA591B7
:103B0000B4918C91822B8C9380916500877F8093F8
:103B100065001092900089E08093910050932E03ED
:103B200040932D0320932C0380E00E94CE1180EF60
:103B300093E09093330380933203F999FECF80EFA3
:103B400093E00E946F3024EF33E0309333032093EF
:103B500032036F3472448E449341B9F5F999FECF24
:103B60004AE050E064EF73E080E493E00E94573055
:103B7000C0913203D09133032A96D0933303C0937C
:103B80003203F999FECFCE010E9475308C01229646
:103B9000D0933303C09332030E942B1180179107F7
:103BA000A1F482E090E0909331038093300310926F
:103BB0002F0380915203882341F10E94AE0BDF91C5
:103BC000CF911F910F910C94EB12E2E4F3E088E0A7
:103BD000DF011D928A95E9F780914303807F2BE6F0
:103BE00032EF4AED20934003309341034093420368
:103BF000836080628093430381E090E0909331037F
:103C00008093300380932F03D4CF0E94A90BD7CF8A
:103C10006F927F929F92AF92BF92CF92DF92EF927C
:103C2000FF920F931F93CF93DF93909137039111DE
:103C300003C0882309F4C1C0A0903A0322E0922E69
:103C40009A0C10913B03F0903C036F2C0F2C000C4E
:103C50007708630181E0C81AD108C0913D030C2E9A
:103C6000000CDD0B22E0210FBE0161507109E12C37
:103C7000092DA60181EE97E00E94971680913903E5
:103C8000882331F194E0B92EB10EE2E06E1A71088A
:103C900022974B2DB301CE010E949C1984E08A0D1E
:103CA000B301680F711D87FD7A95615071094B2D25
:103CB000CE010E949C19492DB601CE010E948308B5
:103CC000CE018B0D911D492DB60101970E948308ED
:103CD000D0E0C0E081E1C82E83E0D82E8091360389
:103CE000082E000C990BC817D9070CF04AC0F60132
:103CF00082819381009709F441C0AF2C0F2C000CF6
:103D0000BB0820913D03022E000C330B245F3F4F74
:103D100040913F03042E000C550BC417D50759F5ED
:103D200044E050E0241B350B3093F1072093F0075B
:103D3000B092F307A092F2070E946C1880913F03A3
:103D4000082E000C990BC817D90771F460913D0338
:103D5000062E000C770BEE24E39405E025E0A50188
:103D600081EE97E00E949716F6E0FF0E219684E020
:103D7000C80ED11CB3CF50E040E0D4CFF394F394FD
:103D8000F5CF809138038823B1F040E150E063E241
:103D900077E085E797E00E94433060915203E6E0C8
:103DA0006E9FB0011124695E784F46E050E085E8CF
:103DB00097E00E94433010923703DF91CF911F911B
:103DC0000F91FF90EF90DF90CF90BF90AF909F90BA
:103DD0007F906F9008950F931F93CF93DF938091FF
:103DE0005103882309F44EC082E290E09093F107DA
:103DF0008093F00784E090E09093F3078093F207BC
:103E000086ED98E00E946C1840E86CE270E090E06B
:103E100080E00E949C19CAE0D0E0D093F107C093E3
:103E2000F00780E390E09093F3078093F2078AEC29
:103E300098E00E946C18409148035091490370E04B
:103E400060E02AE081EE97E00E94611AD093F107CA
:103E5000C093F00786E390E09093F3078093F20716
:103E600080EC98E00E946C18209144033091450347
:103E7000409146035091470366E370E08CE490E084
:103E80000E94091B809151030E94081E80915003DB
:103E9000882309F444C00CE010E0D0E0C0E0809139
:103EA0003F03082E000C990B26E530E08C179D0788
:103EB00011F422E530E08091430390E0AE014D5FC4
:103EC0005F4F02C0959587954A95E2F781709927D3
:103ED000C130D10549F11CF0C430D105BCF140918D
:103EE00043034F7050E070E060E03093F10720939F
:103EF000F0071093F3070093F2072AE081EE97E0B2
:103F00000E94611A60E281EE97E00E942A182196D1
:103F10000A5F1F4FC430D10511F610925003DF9194
:103F2000CF911F910F910895892B69F480EB98E050
:103F30003093F1072093F0071093F3070093F207F3
:103F40000E946C18E4CF88EB98E0F2CF892B19F42B
:103F500088EA98E0EDCF8CEA98E0EACFEF92FF9202
:103F60000F931F93CF93DF93F0905103FF2071F0D5
:103F70000E94140EEE24E39400E222E240E258E0B4
:103F800060E270E086E090E00E94B40B80914B0309
:103F90008370C82FD0E011E0209709F010E021973E
:103FA000811102C0C2E0D0E087E08C9FA0018D9F0C
:103FB000500D1124455F574FE12E08E027E067E2DE
:103FC00070E088E090E00E94B40B89E08C9FA00133
:103FD0008D9F500D11244051584F05E029E062E2B9
:103FE00070E085E190E00E94B40B8F2D0E94081EC6
:103FF0008091480390914903892BC9F080913F0338
:10400000811115C080914B0381708093F40720913A
:104010004003309141034091420350E066E270E07A
:1040200088E590E00E942C1881E08093F407DF91EE
:10403000CF911F910F91FF90EF9008952F923F9293
:104040004F925F926F927F928F929F92AF92BF92A8
:10405000CF92DF92EF92FF920F931F93CF93DF9354
:1040600000D01F92CDB7DEB710910F031330B1F51A
:1040700010924C0180914C0120914D01829F202D86
:10408000112490914E01899F902D112430914F0160
:10409000839F802D112433E834BD909597BD91EF17
:1040A000909380002093880080938A00109251039F
:1040B0000F900F900F90DF91CF911F910F91FF9074
:1040C000EF90DF90CF90BF90AF909F908F907F90B8
:1040D0006F905F904F903F902F9008958091510383
:1040E00090910A03992319F00E94081EC1CF8823DA
:1040F00009F20E94E708E0910C03E695E695F0E0EE
:1041000020910B032695269530E080914B01898301
:10411000882309F43AC140914B03469546954630B1
:1041200088F49EE1499FA00111244D5B5C4FB901C9
:1041300067507109EE24E3940FE02FE0CF01079759
:104140000E94B40BE4E5F1E0FB83EA83EA81FB81A2
:10415000808187FD07C0618170E045E08450990B44
:104160000E949C192A813B812E5F3F4F3B832A830B
:104170002857314059F7EAECF1E0FB83EA83EA8102
:10418000FB8180818F7149F0CF010E94960FDC0185
:10419000CB0142E0BD010E949C192A813B812B5F2B
:1041A0003F4F3B832A832A50334049F758E7A52ED7
:1041B00051E0B52EEDEAF1E0FB83EA83D12CC12C6E
:1041C00067EB262E6DE6362E7CE2472E552453945F
:1041D000E4E86E2EE3E07E2EC60165E070E00E940A
:1041E0003334892B09F004C12A813B81295F3F4F79
:1041F0003B832A83245B3140229DC001239D900D87
:10420000329D900D1124849D9001859D300D949DCB
:10421000300D112480910D0390910E03821B930B9E
:10422000B3010E941F344C01F5018181807F69F147
:104230007401F8E6EF1AF1E0FF0AF7FE03C0F1940B
:10424000E194F10822E6E21A21E0F20AA401B501A4
:104250008A819B810E9467101E141F040CF4D7C032
:10426000EA81FB8140814F70F7E04F9FA00111244C
:10427000405E5C4FDC011397CB010397EE24E3947F
:1042800007E027E0BD010E94B40B8FEFC81AD80ADF
:1042900094E0A90EB11CEFE0CE16D10409F09CCF3A
:1042A00060915301462F4295469547704630D0F4B1
:1042B000FEE14F9FA00111244D5B5C4F80915201A4
:1042C000282F221F2227221F6F71660F622B675033
:1042D000770B8F77EE24E3940FE02FE08750990B54
:1042E0000E94B40B0E94D719113009F4C5C008F41C
:1042F000B3C0123009F0BECE30914B033A838981AE
:10430000882309F4D2C0832F3F3108F08EE12EE1DB
:1043100030E0281B3109229FC001239F900D900D92
:1043200011246AE070E00E943334CB012EE243E9AD
:1043300054E068E170E089960E94B20C9A819C3347
:1043400008F498CEE12C07E02BE240E350E06AE26B
:1043500070E081EE97E00E9497168DEF93E027E3DF
:1043600030E03093F1072093F00721E330E0309301
:10437000F3072093F2070E946C1841E060E370E0BD
:104380008BE290E00E94E61074C011111AC04091B7
:104390004B034C3350F48CE390E0841B91096DEF98
:1043A0007FEF0E943334E60FF71FB90163507109A4
:1043B000EE24E39407E027E049E153E0CF010397BF
:1043C000BFCE123091F740914B034051550B449FA3
:1043D000C001459F900D900D112497FD4F96A5E0CB
:1043E00095958795AA95E1F70897E80FF91FDDCF16
:1043F000EA81FB81858182958695877090E00196A0
:10440000880F991F880F991F881A990A0DCF27E0E6
:10441000E216F1040CF039CFF70134E0E316F104B1
:1044200014F0E3E0F0E00E2D000F000F095F2E2FD7
:10443000220F37E0321B232FEE0CFF1CAC014E196C
:104440005F09635071096E0F7F1FEE24E39481EEC4
:1044500097E00E94971619CF80914B0383FF09C004
:1044600020E34FEE54E068E170E088E290E00E94C3
:10447000B20C0E94B51AFECD80910D0390910E03EF
:1044800080312EE0920768F42FE03EE0281B390BC4
:1044900050E040E070E060E088E690E00E94091B98
:1044A000E9CD20E030E0A901F5CF6A81693208F05A
:1044B00068E26051770B28E443E054E08CE190E03F
:1044C0000E94B20CEA81EC3308F4D4CDE12C07E071
:1044D0002BE240E350E06AE270E081EE97E00E9458
:1044E000971687EF93E03BCF2F923F924F925F92C8
:1044F0006F927F928F929F92AF92BF92CF92DF92F4
:10450000EF92FF920F931F93CF93DF93CDB7DEB758
:1045100060970FB6F894DEBF0FBECDBF80910D033C
:1045200090910E0380312EE0920708F0AFC26CE24A
:1045300071E00E941F34892B09F0A8C2862F63E026
:104540000E941334092FE92EF12C87E0989FA001D7
:1045500011244C545E4F588B4F870E94EB2F21E261
:1045600030E040E050E00E94A0306C5F7F4F8F4F02
:104570009F4F362F3295307FAF85B8892C912F70A1
:10458000232B2C9354E096958795779567955A95AC
:10459000D1F7637011968C9111978C7F682B1196CF
:1045A0006C930E94EB2F29E130E040E050E00E9444
:1045B000A0306D5F7F4F8F4F9F4F6F71660F660FFB
:1045C000EF85F88981818378682B61830E94EB2FC6
:1045D00022E030E040E050E00E94A030AF85B88992
:1045E00011968C91119760FB87F911968C930E941C
:1045F000EB2FECE38E2E912CA12CB12CA501940174
:104600000E94A0306C5F7F4F8F4F9F4F6F73EF857D
:10461000F8898281807C682B62830E94EB2FA50140
:1046200094010E94A0306C5F7F4F8F4F9F4F362FB9
:104630003295330F330F307CAF85B88912962C91A9
:1046400012972F73232B12962C931297F2E09695C4
:10465000879577956795FA95D1F76F7013968C913A
:104660001397807F682B13966C930E94EB2FA8E022
:104670008A2E912CA12CB12CA50194010E94A0306E
:10468000862F8295880F807EEF85F88965816F710E
:10469000682B65830E94EB2F25E030E040E050E07E
:1046A0000E94A030862F8F70AF85B8896C91607F93
:1046B000682B6C930E94EB2F29E730E040E050E03C
:1046C0000E94A030645C7F4F8F4F9F4FEF85F88929
:1046D00066830E94EB2FA50194010E94A030862FD3
:1046E0008770AF85B88915966C911597687F682B90
:1046F00015966C930E94EB2F24E030E040E050E0F0
:104700000E94A0306370862F880F880F880FEF8576
:10471000F8896581677E682B658380911003968197
:10472000899FC001112468E770E00E943334162F7E
:10473000611101C011E00E94EB2F24E030E040E065
:1047400050E00E94A03031E0672B682B692B61F5A7
:10475000612F70E090E080E00E948A320E94BA33BC
:1047600020E030E040E85FE30E9404310E945432D0
:104770004B015C0181E090E0A0E0B0E0F2E08F1638
:104780009104A104B1047CF00E94EB2FA5019401D7
:1047900021503109410951090E94A030DC01CB01AF
:1047A0000196A11DB11D382F812F632F0E94133454
:1047B000182F8F706F7097E09E9DF0019F9DF00DF8
:1047C0001124EC54FE4F90819F70923008F0F2C19A
:1047D0008295807F682B648387E08E9D90018F9DFA
:1047E000300D1124F901EC54FE4F868190E0D9017F
:1047F000A854BE4F6C916F7070E00E9433346350C8
:10480000710927543E4FD9018C918770861717067E
:1048100031F028F067708581887F682B658387E099
:104820008E9DF0018F9DF00D1124EC54FE4F808180
:104830008F70813019F0843009F0C1C1123008F452
:10484000BEC10E94EB2F20E230E040E050E00E9429
:10485000A030605E7F4F8F4F9F4FE12FE150FF0BE5
:104860009F01032E000C440B550B0E94A0302830F2
:1048700008F4A3C1283108F027E128502F7087E001
:104880008E9DF0018F9DF00D1124EC54FE4F22956A
:10489000207F83818F70282B2383B5E00B9F8001BD
:1048A0001124000F111F000F111F08581E4F909167
:1048B0000C039695969580910B0386958695280115
:1048C000E4E14E0E511C47E04E9D90014F9D300D8E
:1048D0001124A9014C545E4F5A8349834DE3242E81
:1048E000312CD901AB54BE4FBC83AB83E92FF0E030
:1048F000FE83ED83282F30E038872F83A981BA818A
:10490000CC908C2D82958F701196CC90BC2DB3706D
:10491000CB2EC29490EFC922C82AD12C41018C1809
:104920009D08092C000CAA08BB08D594C7940D2C2F
:10493000000CEE08FF08C814D904EA04FB048CF448
:104940008C189D08AE08BF0841F00E94EB2FA5010E
:1049500094010E94A0304B015C01C80CD91CEA1CD8
:10496000FB1C8C2D8F73F801C080FC2DF07CCF2EAA
:10497000C82AD801CC92EB81FC81808186958695EE
:104980008F71C82ED12C41018C189D08092C000C68
:10499000AA08BB08F3E0CF0ED11C0D2C000CEE08CA
:1049A000FF08C814D904EA04FB048CF48C189D0891
:1049B000AE08BF0841F00E94EB2FA50194010E94B0
:1049C000A0304B015C01C80CD91CEA1CFB1C9C2DBF
:1049D0009295990F990F907CD8018C918F73892BA8
:1049E0008C9382E0F694E794D794C7948A95D1F794
:1049F000BC2DB06FF801B1830E94EB2F20E031E0B5
:104A000040E050E00E94A030D80112966C9350E034
:104A100040E0B8018F8598890E9467106B017C0186
:104A20006D817E816C197D09072E000C880B990B16
:104A30000E948C324B015C016F8178856E197F0971
:104A4000072E000C880B990B0E948C32A501940153
:104A50000E94833120E030E040E053E40E9447337D
:104A60002BED3FE049E450E40E94E23120E030E0E9
:104A700040E05FE30E9404310E945432F8016383F6
:104A80000C5F1F4F0415150509F038CF1A821982E3
:104A90001A861B82B8E72B2EB1E03B2E1DEA412E71
:104AA00011E0512E89819A8165E070E00E943334D3
:104AB000892B09F0A5C0F7E04F0E511C9201245B31
:104AC000314047EB5DE6249FC001259F900D349F48
:104AD000900D1124ACE2B1E08A9F90018B9F300DC4
:104AE0009A9F300D112480910D0390910E03821B2B
:104AF000930B64E873E00E941F343C01D1011196CE
:104B00008C91982F907FD1F0B1ED6B16B2E07B06BF
:104B10001CF08F70F101818380910F03813071F45B
:104B2000C3010697853C924008F478C06114710473
:104B300029F463E089EA95E00E945216E981FA813E
:104B40003196FA83E983F4E02F0E311C29813A81F2
:104B50002F30310509F0A6CF3A85332331F06AE0D2
:104B600070E088EC90E00E94FB114B81411108C07D
:104B700081E020910D0330910E0320313E4008F476
:104B800080E060960FB6F894DEBF0FBECDBFDF9118
:104B9000CF911F910F91FF90EF90DF90CF90BF903A
:104BA000AF909F908F907F906F905F904F903F90CD
:104BB0002F9008956295607F0DCE20E060CE0E9418
:104BC000EB2F47E04E9D90014F9D300D1124A90120
:104BD0004C545E4F6A0124E030E040E050E00E9417
:104BE000A0306F5F7F4F8F4F9F4F6295607FD601E0
:104BF00013968C9113978F70682B13966C934DCEF0
:104C0000F201858182958695877090E00196880FE4
:104C1000991F880F991F681A790A70CFA301B101F3
:104C2000C2010E9467104B015C0178876F839E83ED
:104C30008D838C01035011099B0123503109E4E558
:104C4000F1E0AB014C5F5F4FBC016C5F7F4FD10166
:104C50001196FC908F2D807F09F4B6C0B1E0E83743
:104C6000FB0709F4C7C0808187FD1EC0B18190E0B9
:104C700082179307CCF084179507B4F48B2F90E03C
:104C8000801791078CF08617970774F480E880836B
:104C90008F2D807F80519F2D9F70F92EF82AD10192
:104CA0001196FC92B1E0BA873296D1CF433009F425
:104CB00078C0443009F042CFF201F481F295FF70E0
:104CC000F987D10113961C91F12CE12CEF2FF0E024
:104CD000F88BEF872F853889E216F3060CF06CC04D
:104CE00000320CF069C0101644F4202F412F6D8162
:104CF0007E818F8198850E94610E3FEFE31AF30A4F
:104D00000F5FE8CFD20114960C9102950F7010E05E
:104D1000FE85E3E0FE02F0011124F88BEF87F7FF38
:104D200003C03196F88BEF872F8538893595279505
:104D3000388B2F87C80195958795281B2987D12CFB
:104D4000C12CC016D1060CF0F9CE398530320CF0EA
:104D5000F5CE131644F4232F4F2D6D817E818F8164
:104D600098850E94610E4FEFC41AD40A59855F5F7F
:104D70005987E7CFEE85F3E0EF029001112437FF6A
:104D800002C02F5F3F4F35952795D20114960C91A5
:104D900002950F70F1014381B501C4010E948B0E91
:104DA000CDCED20114960C9102950F702F85220F53
:104DB000BE85B01B2B0FCBC0D1011396EC9013977F
:104DC000DE0C1396DC92BACE62E08DE995E00E948B
:104DD0005216D2018C918F700E94570F882DA0FA25
:104DE00087F980935201C501969587958F718093BD
:104DF0005301A4CEBB81BF5FBB83F201F581F9876C
:104E00002F2F2770D10112968C91860D972D911D11
:104E1000F201668170E00E9433342D5F622F70E0F2
:104E20000E941F346F87892B09F088CEEF85EB87AE
:104E3000D20114961C911F70E11708F07FCE80916B
:104E400010038C5FB985B695B695B695B370B80F5B
:104E5000BE870B2F60910C036695669570E068190C
:104E60007909072E000C880B990B0E948C326B017C
:104E70007C0160910B036695669570E06A197B0969
:104E8000072E000C880B990B0E948C32A70196010B
:104E90000E94833120E030E040E053E40E94473339
:104EA0002BED3FE049E450E40E94E23120E030E0A5
:104EB00040E05FE30E9404310E945432F62EF2017A
:104EC000E380E294EFE0EE22F985F170FC871D8625
:104ED0008C859D85880F991F019798E09E0D989F5E
:104EE000D02C1124D2014C91BB85B1111AC0F10113
:104EF000F382842F8F708430A1F4123090F0812FD0
:104F00008150990B9C015D2D5203C001539F900D60
:104F1000112497FD019695958795AF2DA81BF1015A
:104F2000A3834F70423009F425CF08F0BFCE44234D
:104F300009F4E8CE413009F001CED20114960C916B
:104F400002950F70BF85B1700B1BED2C2E854F2D78
:104F500023CFCF93DF9380912F03882309F45BC085
:104F60008091300390913103019709F057C080EF91
:104F700093E09093330380933203F999FECF4FE48B
:104F800052E46EE473E180EF93E00E9493308091ED
:104F9000320390913303049690933303809332034A
:104FA000F999FECF60913203709133034AE050E0EB
:104FB00080E493E00E947B30C0913203D0913303B0
:104FC0002A96D0933303C09332030E942B11F99990
:104FD000FECFBC01CE010E949B30809132039091A4
:104FE000330302969093330380933203C0915203AC
:104FF00082E090E00E946730C81729F06C2F82E0B1
:1050000090E00E94853082E090E09093310380939D
:10501000300310922F03DF91CF91089584EF93E036
:10502000BBCF0E9470120E94A92710920A0383E04E
:1050300080930F03089580914B01882321F0809184
:105040004B038C33B8F10E94C70E80915301982F07
:10505000929596959770963040F49F5F9295990F30
:10506000907E8F71892B809353010E94CE0F0E94F6
:10507000742280910D0390910E03803E20E19207EF
:1050800028F4019690930E0380930D0380914B03B7
:105090008C3380F087FF03C0885080934B0384E0FB
:1050A0000E947108882369F080914B01882331F0B8
:1050B0000E94C81C81E08093510308950E9411282A
:1050C000F9CF88E00E9471088823A1F30E9484131D
:1050D000F1CF0E94C70E0E94D40E80915301982FE9
:1050E000929596959770963040F49F5F9295990FA0
:1050F000907E8F71892B809353010E94CE0F8093F5
:105100004B010E94742220910D0330910E032F5FFA
:105110003F4F30930E0320930D0340914403509171
:10512000450360914603709147034F5F5F4F6F4F98
:105130007F4F40934403509345036093460370931D
:10514000470391E090932F0390914B0191110AC076
:1051500081111BC088E00E947108882391F00E9491
:1051600084130FC061E086E695E00E94521685E048
:105170000E94570F0E94A92710924B0382E0809350
:105180000F0381E080935103089561E08FE495E07F
:105190000E94521680914303806880934303EACFB4
:1051A000CF93C0914B03CC33D8F00E94C70E0E941E
:1051B000D40EC837A9F48091480390914903019611
:1051C0009093490380934803C1E0C0932F030E944A
:1051D000A927C0930F0381E080935103CF910895D5
:1051E00088E00E9471088823B1F30E948413F3CFF2
:1051F0001F920F920FB60F9211248F939F9380915D
:10520000E1009091E100937F9093E10083FF0FC054
:105210001092E90091E09093EB001092EC0092E381
:105220009093ED001092720398E09093F00082FF4B
:1052300022C093E09093E9009091F200992319F035
:105240009AE39093E80090916303992341F0909141
:105250006303915090936303911101C05D9A909103
:105260007103992341F090917103915090937103D0
:10527000911101C0289A84FF18C08091E2008E7EAF
:1052800081608093E2008091E1008F7E8093E10055
:10529000809164038E7E8061809364039F918F91DF
:1052A0000F900FBE0F901F90189580FFF7CF809141
:1052B000E2008E7E80618093E2008091E1008E7E2C
:1052C0008093E100809164038E7E8160E5CF1F9220
:1052D0000F920FB60F921124CF92DF92EF92FF92AE
:1052E0000F931F932F933F934F935F936F937F93EE
:1052F0008F939F93AF93BF93EF93FF93CF93DF93DE
:10530000CDB7DEB76C97DEBFCDBF1092E9008091BC
:10531000E80083FF25C068E0CE0145960E94820A1E
:1053200082EF8093E8008D8987FF39C09091E80073
:1053300090FFFCCF982F907609F034C19E894F8959
:10534000588D2F89F88C911131C0803861F580918A
:1053500062038093F1001092F1008EEF8093E800D9
:105360006C960FB6F894DEBF0FBECDBFDF91CF9124
:10537000FF91EF91BF91AF919F918F917F916F912D
:105380005F914F913F912F911F910F91FF90EF905F
:10539000DF90CF900F900FBE0F901F9018959EEF4B
:1053A0009093E800C7CF1092F100D5CF913059F417
:1053B0008111D3CF4130510581F6809162038D7FF9
:1053C00080936203CACF933049F48111C6CF413034
:1053D000510519F6809162038260F2CF953041F455
:1053E0008091E80080FFFCCF20682093E300B5CFD8
:1053F000963009F0A9C00B8D1C8D22E01092E900B7
:105400001092600310925F03F2122EC010925E039E
:1054100010925D030E94510A1F8299E09983FA82DB
:1054200091E09E8390EA98879AEF998720915F0395
:1054300030916003275F3F4F3C832B838D83109215
:10544000E9001092600310925F0310935E030093D3
:105450005D0349E050E0BE016F5F7F4F80E00E9436
:105460002B0A0E94510A79CF10935E0300935D03CB
:105470000E943509DC0112960D911C910115110550
:1054800009F451C1D801ED91FC910480F581E02D22
:10549000BE016B5E7F4FC8010995009709F03EC1C0
:1054A000F80100851185EACFF3E0FF120EC08F8965
:1054B000882309F440C0823061F440E867E083E665
:1054C00090E10E94F809811148CF81E28093EB00BE
:1054D00047CF813029F440E86BE087E590E1F1CFD8
:1054E000833099F70E943509DC011296ED90FC900B
:1054F0008E010F5F1F4F6801E114F10479F0D701AD
:10550000ED91FC910680F781E02DB801C701099566
:10551000080F111DF701E084F184EECFD8011C9231
:10552000F60101900020E9F73197BF016C197D0960
:1055300040E0C601C6CF61E470E1FB01449150E058
:1055400080E80E942B0A09CF973009F4BECF98302B
:1055500021F481E08093F10000CF993009F0FDCE75
:10556000837009F0B2CFE9E1F1E081E031E096E348
:105570002191222371F08093E9003093EB00DF0149
:1055800011972C912093EC009093ED008F5F873062
:1055900079F78EE78093EA001092EA008F89809372
:1055A0007203DBCE8B8D9C8D1092E900109260030C
:1055B00010925F0390935E0380935D03898D811148
:1055C00092C08E899D89913A49F4813209F07DCF4C
:1055D00047E050E068E071E080E0B3CF913209F03D
:1055E00074CF833269F48F89988DB0E0A0E0809306
:1055F000040190930501A0930601B0930701ADCE7D
:10560000803269F48091E80082FFFCCF67E088E097
:1056100091E00E94820A8BEF8093E8009ECE823256
:1056200009F09BCE8F8980930F01EEEFFFE7859104
:1056300094918B3F9C4D51F1E0E0F8E0809108019E
:1056400090910901A0910A01B0910B01803B944017
:10565000A105B105F1F480910F0180FD1AC0EE3F64
:105660008AE0F80789F587E797E79183808380913F
:1056700060008093610388E19BE00FB6F894A895E1
:10568000809360000FBE9093600067CEEEEFFAE06B
:10569000D5CF808191818737974709F05ECEA89555
:1056A00080916000886180936000809161038093A5
:1056B0006000EE3F2AE0F20789F08091FE0A9091A7
:1056C000FF0A9183808349CE808191818737980733
:1056D00051F29093FF0A8093FE0AC5CF1092FF0A01
:1056E0001092FE0A3ACE0E943509DC0112960D9105
:1056F0001C910115110509F4E8CED801ED91FC913A
:105700000190F081E02DBE016B5E7F4FC8010995CD
:10571000811123CEF80100851185EBCF18161906EB
:105720000CF41BCED2CEF1E0FF12BECE65E470E1E8
:1057300004CF1F920F920FB60F9211242F933F9315
:105740008F939F93AF93BF93809158039091590388
:10575000A0915A03B0915B033091530323E0230FD0
:105760002D3758F50196A11DB11D20935303809349
:10577000580390935903A0935A03B0935B0380910D
:10578000540390915503A0915603B091570301968D
:10579000A11DB11D8093540390935503A09356030C
:1057A000B0935703BF91AF919F918F913F912F91EC
:1057B0000F900FBE0F901F90189526E8230F0296AA
:1057C000A11DB11DD2CF1F920F920FB60F921124BF
:1057D0002F933F934F935F936F937F938F939F93F9
:1057E000AF93BF93EF93FF9380918403882329F1B4
:1057F00080917A03811121C08091850381111DC0A0
:105800006091800370918103809182039091830362
:105810002091490130E050E040E00E94D2306230F7
:1058200071058105910548F490912C03E0912D03B9
:10583000F0912E038081892780838091800390914D
:105840008103A0918203B0918303892B8A2B8B2B38
:10585000E9F08091800390918103A0918203B0913F
:1058600083030197A109B109809380039093810379
:10587000A0938203B0938303892B8A2B8B2B31F463
:1058800080918903882399F00E946C15FF91EF9114
:10589000BF91AF919F918F917F916F915F914F9148
:1058A0003F912F910F900FBE0F901F90189580E0A1
:1058B0000E94CE11EBCF1F920F920FB60F921124C0
:1058C0002F933F934F935F936F937F938F939F9308
:1058D000AF93BF93EF93FF9380917F03882309F4E5
:1058E00072C080917B0390917C03A0917D03B09165
:1058F0007E03892B8A2B8B2B09F451C08091850361
:1059000081111DC060917B0370917C0380917D03A8
:1059100090917E032091480130E050E040E00E94E9
:10592000D230623071058105910548F490912903C8
:10593000E0912A03F0912B03808189278083809155
:105940007B0390917C03A0917D03B0917E03892B12
:105950008A2B8B2B99F080917B0390917C03A091F3
:105960007D03B0917E030197A109B10980937B0368
:1059700090937C03A0937D03B0937E03FF91EF91FE
:10598000BF91AF919F918F917F916F915F914F9157
:105990003F912F910F900FBE0F901F90189510926E
:1059A0007A0310927F0380916F008D7F80936F0048
:1059B00080912903E0912A03F0912B039081809537
:1059C00089238083DBCF809185038111D7CF6091BC
:1059D0007B0370917C0380917D0390917E032091E5
:1059E000480130E050E040E00E94D2306230710562
:1059F0008105910518F690912903E0912A03F09111
:105A00002B0380818927DDCF0F931F93CF93DF93E3
:105A10008C0181E090E00E94673080FF31C08AE015
:105A200090E00E9467309FEF980F9E3F48F522E379
:105A300030E0D80150963C932E931F9728E330E036
:105A400052963C932E935197CBE0D0E0D801ED9144
:105A5000FC910190F081E02D682FC8010995CE01DD
:105A60000E9467302196C131D10581F70E946108FB
:105A700088EE93E0DF91CF911F910F910C94990BD9
:105A8000DF91CF911F910F91089504970C94042DED
:105A9000EBE8F7E01382128288EE93E0A0E0B0E03A
:105AA00084839583A683B78383E291E09183808387
:105AB0008FEF9FEF95878487EBEDF7E011821082DF
:105AC0001382128280E8848380E48583E1EEF7E02C
:105AD000138212821186128680E1838710861782D4
:105AE0001586108A1786128A118A81E0838B148AA0
:105AF000858B168A85E391E09183808383E491E02E
:105B0000958384830895789484B5826084BD84B538
:105B1000816084BD85B5826085BD85B5816085BDA8
:105B200080916E00816080936E0010928100809160
:105B300081008260809381008091810081608093E8
:105B4000810080918000816080938000809191002D
:105B50008260809391008091910081608093910098
:105B6000809190008160809390008091C10084605A
:105B70008093C1008091C10082608093C1008091B8
:105B8000C10081608093C1008091C30081608093D7
:105B9000C3008091C00082608093C0008091C200E9
:105BA00081608093C20080917A00846080937A0043
:105BB00080917A00826080937A0080917A0081607F
:105BC00080937A0080917A00806880937A001092A6
:105BD000720310926203109264038091D700816077
:105BE0008093D70080EA8093D80089B5806189BD11
:105BF00089B5826089BD09B400FEFDCF61E070E027
:105C000080E090E00E94E10A8091D8008F7C806162
:105C10008093D8008091E000807F8093E0008091A5
:105C2000E1008E7E8093E1008DE08093E200559A42
:105C3000209A81EC80937C0085B1806F85B984B116
:105C4000877E84B984B1876E84B95E9A5F988AB181
:105C5000806D8AB9769A6E9881B3806F81BB89987E
:105C600080B38D7080BB80E58CBD81E08DBD85E00B
:105C700090E00E94990B5F9A85E090E00E94990B5A
:105C80005E985C98EFEDFFE084918EBD00000DB44E
:105C900007FEFDCF31968FE0ED3EF807A9F75C9A3D
:105CA00081E8809364008091650081608093650045
:105CB0000E9461080E949E0B87FF15C05C9885EAD0
:105CC0008EBD00000DB407FEFDCF5C9A2E982F9874
:105CD0002D988091640080628093640081E083BF8E
:105CE000889513BEFCCF0E949E0B82FF46C02D9864
:105CF0000E949E0B84788438D9F42D9A88EC90E029
:105D00000E94990B2F9882E090E00E9467308F3FAD
:105D100029F06FEF82E090E00E94853084EF91E0FF
:105D20000E94990B2F9A0E949E0B84788438D9F395
:105D30000E949E0B84718431D9F42D9A88EC90E0F6
:105D40000E94990B2E9882E090E00E946730882391
:105D500029F060E082E090E00E94853084EF91E0DD
:105D60000E94990B2E9A0E949E0B84718431D9F364
:105D700088EC90E00E94990BB6CF2D9A82E090E0DB
:105D80000E946730882391F10E94AE0B80E18093DE
:105D9000EC0710925C03EDEEFFE085919491FC011D
:105DA0000995FF24F394D6E000E010E0EE24E3949C
:105DB0008FB7F894409158035091590360915A035A
:105DC00070915B038FBF8091ED07F42FF81B8F2F2D
:105DD0009091EE07992369F0F093EF071092EE0788
:105DE0000115110529F30E940000E2CF0E94A90BC2
:105DF000CDCF9091EC07F91738F48F5F891780F7B2
:105E0000F3BE889513BEECCFE092EE074093ED070A
:105E10008091E8079091E90701969093E9078093B4
:105E2000E8078091F9078093F8070E949E0B809302
:105E3000F907E0915C03DE9FF0011124E151F04F7E
:105E400085919491FC010995C82FE0915C03DE9F38
:105E5000F0011124EF50F04F85919491FC010995C8
:105E60000E94610880915C03C81709F4B9CFC09300
:105E70005C03DC9FF0011124E351F04F8591949174
:105E8000FC010995ADCF8F929F92AF92BF92CF92B6
:105E9000DF92EF92FF92CF93DF93EC0168817981DB
:105EA0008A819B81611571058105910521F464E268
:105EB00079ED8BE597E02DE133EF41E050E00E9472
:105EC000A03049015A019B01AC01A7EAB1E40E944C
:105ED000BF306B017C01ACEEB4EFA50194010E94D0
:105EE000CD30DC01CB018C0D9D1DAE1DBF1DB7FF5C
:105EF00003C00197A109B04888839983AA83BB8313
:105F00009F77DF91CF91FF90EF90DF90CF90BF9080
:105F1000AF909F908F9008950E94432F089580E145
:105F200091E00E94432F0895B0E0A0E0809310011B
:105F300090931101A0931201B093130108958F92D1
:105F40009F92AF92BF92CF92DF92EF92FF92CF9348
:105F5000DF93EC01688179818A819B8161157105EC
:105F60008105910521F464E279ED8BE597E02DE15F
:105F700033EF41E050E00E94A03049015A019B01FB
:105F8000AC01A7EAB1E40E94BF306B017C01ACEE2A
:105F9000B4EFA50194010E94CD30C60ED71EE81EB5
:105FA000F91EF7FE06C081E0C81AD108E10880E8B2
:105FB000F80AC882D982EA82FB82C701B6019F77BC
:105FC000DF91CF91FF90EF90DF90CF90BF90AF9097
:105FD0009F908F9008958F929F92AF92BF92CF9291
:105FE000DF92EF92FF926091140170911501809100
:105FF000160190911701611571058105910521F434
:1060000064E279ED8BE597E02DE133EF41E050E07C
:106010000E94A03049015A019B01AC01A7EAB1E4FA
:106020000E94BF306B017C01ACEEB4EFA50194017E
:106030000E94CD30C60ED71EE81EF91EF7FE06C020
:1060400081E0C81AD108E10880E8F80AC09214017A
:10605000D0921501E0921601F0921701C701B60126
:106060009F77FF90EF90DF90CF90BF90AF909F9081
:106070008F90089560931401709315018093160119
:10608000909317010895FB01DC0102C005900D9269
:1060900041505040D8F70895FC0105906150704080
:1060A0000110D8F7809590958E0F9F1F0895DC0101
:1060B000CB01FC01F999FECF06C0F2BDE1BDF89A13
:1060C000319600B40D9241505040B8F70895F999B7
:1060D000FECF92BD81BDF89A992780B50895A6E1BB
:1060E000B0E044E050E00C945930A8E1B0E042E068
:1060F00050E00C945930DC01CB0103C02D910E947B
:10610000863041505040D0F70895262FF999FECFA0
:106110001FBA92BD81BD20BD0FB6F894FA9AF99AC4
:106120000FBE01960895242F0E948630252F0E94CD
:1061300086300C949B300E948530272F0C9486303B
:10614000052E97FB1EF400940E94B73057FD07D030
:106150000E94D23007FC03D04EF40C94B730509517
:106160004095309521953F4F4F4F5F4F0895909543
:106170008095709561957F4F8F4F9F4F08950E9436
:10618000F430A59F900DB49F900DA49F800D911D9C
:1061900011240895B7FF0C94BF300E94BF30821BBA
:1061A000930B0895A1E21A2EAA1BBB1BFD010DC083
:1061B000AA1FBB1FEE1FFF1FA217B307E407F507B7
:1061C00020F0A21BB30BE40BF50B661F771F881F93
:1061D000991F1A9469F760957095809590959B0129
:1061E000AC01BD01CF010895A29FB001B39FC001D2
:1061F000A39F700D811D1124911DB29F700D811DF3
:106200001124911D08955058BB27AA270E941B31C5
:106210000C9405330E94F73238F00E94FE3220F0D1
:1062200039F49F3F19F426F40C94CD320EF4E09526
:10623000E7FB0C94C732E92F0E94163358F3BA17C4
:10624000620773078407950720F079F4A6F50C948C
:1062500038330EF4E0950B2EBA2FA02D0B01B901A7
:1062600090010C01CA01A0011124FF27591B99F0CC
:10627000593F50F4503E68F11A16F040A22F232FD8
:10628000342F4427585FF3CF469537952795A79528
:10629000F0405395C9F77EF41F16BA0B620B730BCF
:1062A000840BBAF09150A1F0FF0FBB1F661F771F40
:1062B000881FC2F70EC0BA0F621F731F841F48F4F5
:1062C000879577956795B795F7959E3F08F0B0CF7E
:1062D0009395880F08F09927EE0F97958795089565
:1062E0000E94F73260F080E891E009F49EEF0E948E
:1062F000FE3228F040E851E071F45EEF0CC00C94DF
:10630000CD320C943833E92FE0780E94163340F3F5
:10631000092E052AB1F3261737074807590738F021
:106320000E2E07F8E02569F0E025E0640AC0EF636F
:1063300007F8009407FADB01B9019D01DC01CA01ED
:10634000AD01EF930E94F9310E9405330E94B331F1
:106350005F91552339F02BED3FE049E450FD49ECC6
:106360000C9404310895DF93DD27B92FBF7740E8FF
:106370005FE31616170648075B0718F4D92F0E942B
:106380003F339F938F937F936F930E94FA33ECEA8E
:10639000F0E00E94D0320E9405332F913F914F913F
:1063A0005F910E945A33DD2351F09058A2EA2AED02
:1063B0003FE049EC5FE3D0785D270E941B31DF911D
:1063C0000C9405330E94F6310C9405330E94FE3282
:1063D00058F00E94F73240F029F45F3F29F00C9406
:1063E000C73251110C9439330C94CD320E941633BC
:1063F00068F39923B1F3552391F3951B550BBB27F4
:10640000AA2762177307840738F09F5F5F4F220F38
:10641000331F441FAA1FA9F335D00E2E3AF0E0E82F
:1064200032D091505040E695001CCAF72BD0FE2F79
:1064300029D0660F771F881FBB1F2617370748070D
:10644000AB07B0E809F0BB0B802DBF01FF279358C5
:106450005F4F3AF09E3F510578F00C94C7320C9490
:1064600039335F3FE4F3983ED4F38695779567958B
:10647000B795F7959F5FC9F7880F911D96958795FA
:1064800097F90895E1E0660F771F881FBB1F621719
:1064900073078407BA0720F0621B730B840BBA0BD7
:1064A000EE1F88F7E09508950E945B326894B11161
:1064B0000C94393308950E941E3388F09F5798F04A
:1064C000B92F9927B751B0F0E1F0660F771F881FF9
:1064D000991F1AF0BA95C9F714C0B13091F00E9413
:1064E0003833B1E008950C943833672F782F88271C
:1064F000B85F39F0B93FCCF3869577956795B3953A
:10650000D9F73EF490958095709561957F4F8F4FA8
:106510009F4F0895E89409C097FB3EF490958095AD
:10652000709561957F4F8F4F9F4F9923A9F0F92F59
:1065300096E9BB279395F695879577956795B795D7
:10654000F111F8CFFAF4BB0F11F460FF1BC06F5FBD
:106550007F4F8F4F9F4F16C0882311F096E911C0CF
:10656000772321F09EE8872F762F05C0662371F0F0
:1065700096E8862F70E060E02AF09A95660F771F04
:10658000881FDAF7880F9695879597F9089597F9F8
:106590009F6780E870E060E008959FEF80EC0895C9
:1065A000DF93CF931F930F93FF92EF92DF927B01C4
:1065B0008C01689406C0DA2EEF010E945A33FE0166
:1065C000E894A5912591359145915591A6F3EF0158
:1065D0000E941B31FE019701A801DA9469F7DF9050
:1065E000EF90FF900F911F91CF91DF9108950024BC
:1065F0000A941616170618060906089500240A9428
:1066000012161306140605060895092E0394000CAD
:1066100011F4882352F0BB0F40F4BF2B11F460FF3C
:1066200004C06F5F7F4F8F4F9F4F089557FD905865
:10663000440F551F59F05F3F71F04795880F97FB46
:10664000991F61F09F3F79F0879508951216130600
:106650001406551FF2CF4695F1DF08C0161617062F
:106660001806991FF1CF8695710561050894089564
:10667000E894BB2766277727CB0197F908959B01FC
:10668000AC0160E070E080E89FE30C94E2310E948E
:106690005A330C9405330E94F73238F00E94FE32D0
:1066A00020F0952311F00C94C7320C94CD321124B4
:1066B0000C9439330E94163370F3959FC1F3950FF4
:1066C00050E0551F629FF001729FBB27F00DB11D76
:1066D000639FAA27F00DB11DAA1F649F6627B00D06
:1066E000A11D661F829F2227B00DA11D621F739FEF
:1066F000B00DA11D621F839FA00D611D221F749FFD
:106700003327A00D611D231F849F600D211D822F43
:10671000762F6A2F11249F5750409AF0F1F088236A
:106720004AF0EE0FFF1FBB1F661F771F881F915097
:106730005040A9F79E3F510580F00C94C7320C944D
:1067400039335F3FE4F3983ED4F3869577956795A8
:10675000B795F795E7959F5FC1F7FE2B880F911DC1
:106760009695879597F9089519F416F40C94CD32FF
:106770000C94FE330E941E33B8F39923C9F3B6F389
:106780009F57550B87FF0E940C340024A0E640EA77
:10679000900180585695979528F4805C660F771F76
:1067A000881F20F026173707480730F4621B730B49
:1067B000840B202931294A2BA6951794079420256C
:1067C00031254A2758F7660F771F881F20F02617B4
:1067D0003707480730F4620B730B840B200D311D13
:1067E000411DA09581F7B901842F9158880F969586
:1067F000879508959B01AC010C9447339F3F31F07E
:10680000915020F4879577956795B795880F911DDE
:106810009695879597F9089591505040660F771F88
:10682000881FD2F70895991B79E004C0991F961725
:1068300008F0961B881F7A95C9F780950895AA1BC2
:10684000BB1B51E107C0AA1FBB1FA617B70710F05B
:10685000A61BB70B881F991F5A95A9F7809590958D
:10686000BC01CD01089597FB072E16F4009407D0C4
:1068700077FD09D00E941F3407FC05D03EF49095A7
:1068800081959F4F0895709561957F4F0895EE0F04
:10689000FF1F0590F491E02D099481E090E0F894B9
:0868A0000C945234F894FFCF70
:1068A8005401CA01FFFFFFFF00E1000000000000E3
:1068B800010000000100000000C18081000000000C
:1068C8000000004909140B6A095F09B0096E098CB8
:1068D800090000000027178F0A99199819042DFC40
:0668E800FF0000452D0039
:00000001FF
